:106BD000011900000501013C0200000301FA040054
:106BE000FA0500030A0A5A0B001E0C00FA0D0003F6
:106BF0000E00040F0164100096120132130AFA14F9
:106C0000010215000217010A1801FA1905321A01CA
:106C10000A1B01FA1C05321FFFFF20FFFF23011E84
:106C20002400642A00FA2B00FA2C50782D003D2E07
:106C300000462F001E30006432507833000034329A
:106C4000FA350164360164370150380A643C006447
:106C50003E003C3F000140FFFF411450420A5A43AE
:106C60000AC84405324500B44600FA470178480294
:106C7000034C00FA4EFFFF500808510596520A32A5
:106C8000530B46540A9656010257054658000259BE
:106C90000A465A32FA5B010A5C0A325E000A5F0059
:106CA000FE61FFFF64021C66000267FFFF6A0A3C88
:106CB0006B00006C3296730000740000780132792A
:106CC00001327EFFFF81FFFF84FFFF8500AF86005A
:106CD000018700FA89010A8A00009900009D0A963E
:106CE0009E00019FFFFFA0FFFFFAFAFA00000501D6
:106CF000013C0200000301FA0400FA0500030A0A3D
:106D00005A0B001E0C00FA0D00030E00040F016464
:106D1000100096120132130AFA140102150000172E
:106D2000010A1801FA1905321A010A1B01FA1C0599
:106D3000321FFFFF20FFFF23011E2400642A00FAF8
:106D40002B00FA2C50782D003D2E00462F001E30CF
:106D500000643250783300003432FA350164360171
:106D600064370150380A643C00643E003C3F000137
:106D700040FFFF411450420A5A430AC844053245B5
:106D800000B44600FA47013C4802024C00FA4EFFAC
:106D9000FF500808510596520A32530B46540A9682
:106DA000560101570546580001590A465A32FA5B06
:106DB000010A5C0A325E000A5F00FE61FFFF6403A5
:106DC0001C66000267FFFF6A0A3C6B00006C32968B
:106DD0007300007400007801327901327EFFFF8178
:106DE000FFFF84FFFF85FFFF86FFFF87FFFF89010D
:106DF000028A00009900009D0A969E00019FFFFFF5
:106E0000A0FFFFFAFAFA0065006F00790083008D99
:106E1000009700A100AC00B600C000CA00D400DE9C
:106E200000E800F200580060006800700078008000
:106E300000880090009800A000A800B000B800C131
:106E400000C800D000D800DF00E600EE00F60041E8
:106E50000047004D00530059005F0065006C007151
:106E60000077007D00830089008F0095009B00A2C1
:106E700000A700AC00B200B900C000C500CA00D233
:0A6E800000D500DD00E100E700EF9F
:103A390090005FE0D3940440149007D0E0FEA3E027
:103A4900FF906BD2126FC3E493F59980129007D05F
:103A5900E0FEA3E0FF906CEC126FC3E493F599903C
:103A690007D0E0FEA3E0FF906BD0E493FC740193D0
:103A7900FDEFB50507EEB50403754D009007D012AB
:103A89006FAA2285F97385FA747E017F00E57412A5
:103A99006F9CE5732FFF50010E8E5A8F5B90001BB0
:103AA900E0FCA3E0FDEF2DFDEE3CFC8C5C8D5D227E
:103AB90075A71085F97385FA747E017F00E5741284
:103AC9006F9CE5732FFF50010E8E5A8F5B90001B80
:103AD900E0FCA3E0FDEF2DFDEE3CFC8C5C8D5D224E
:103AE900E55DF5FBE55CF5FCD29322E55DF5E9E5DD
:103AF9005CF5EAD29422E55DF5EBE55CF5ECD29153
:103B090022E55DF5EDE55CF5EED29222E55DF5FB8A
:103B1900E55CF5FCD28722E55DF5E9E55CF5EAD2DD
:103B29009022E55DF5EBE55CF5ECE5B54410F5B5FE
:103B390022E55DF5EDE55CF5EEE5B54420F5B52248
:103B4900AE5AAF5B74068E048F05FF126F8C8C5CC6
:103B59008D5DAE5AAF5B74068E048F05FF126FB789
:103B69008C5A8D5BE55B455A60137406C3955BFF00
:103B7900E4955AFE8E5A8F5B785C126FF0E573A854
:103B89005CB80015D3955D4010E573C3955DFFE4FE
:103B9900955CFE8E5C8F5D8010E573243CC3955D5A
:103BA900FFE4955CFE8E5C8F5DAE5CAF5D743B6F30
:103BB9004E6006743C6F4E701AAE5CAF5D743B6F1D
:103BC9004E70057573018003757302755D3A755CF6
:103BD900008003757300229000A0E0B40104C210B4
:103BE9008002D2109000A1E0B40104C2118002D277
:103BF900119000DEE075F0DCA4FFAEF0740A8E04CB
:103C09008F05FF126F8C9007C6ECF0A3EDF0A20DA3
:103C1900401674038C068D07126F9C7401120039CB
:103C29009007C4EEF0A3EFF07E017F0090009CE0C6
:103C3900126F9C9000DFE08E048F05FF126F8C7469
:103C49000AFF126F8C8D609000E8E075F0DCA4FF2C
:103C5900AEF0740A8E048F05FF126F8C9007CAECC0
:103C6900F0A3EDF09000EAE060139000EAE0F5F0CF
:103C7900741684FF7E00EF9007D8F0800674649074
:103C890007D8F09000E0E0900084F090012AE090DD
:103C9900006EF09000B9E0900070F09000E2E090C2
:103CA9000071F090008EE0900072F0900114E090A5
:103CB9000077F0900178E0900078F0900179E09039
:103CC9000079F090017AE090007AF0A22DB34016C5
:103CD900900178E0700C900179E0700690017AE02B
:103CE90060028002C22D74E3900083F09000C9E065
:103CF900B40B0874E3900083F0805A9000C9E0B4D3
:103D090019129000DFE0906DF112008CE49390009D
:103D190083F080419000C9E0B41E129000DFE0906A
:103D29006E0F12008CE493900083F080289000C9F4
:103D3900E0B428129000DFE0906E3912008CE49311
:103D4900900083F0800F9000C9E0B446089000C04D
:103D5900E0900083F09000F9E0FE9000C7E06E600B
:103D69000A9000C7E09000F9F0D22C900087E0FE9D
:103D79009000C6E0B50633900088E0FE9000F2E0BE
:103D8900B50627900089E0FE9000E4E0B5061B9097
:103D9900008BE0FE900099E0B5060F90008AE0FEE6
:103DA9009000D4E06E7003023F6690005FE0C39418
:103DB9000550087402900115F0801C9000D4E0644D
:103DC9000360069000F2E060087406900115F08027
:103DD90006740A900115F09000D4E0B4030890002D
:103DE900F2E064026002800674009000F2F0900034
:103DF90099E0B4010674009000FFF0900099E0B4D6
:103E0900020674009000E4F0900099E0B40306748F
:103E1900009000F1F09000C6E0601474199000ADB4
:103E2900F074009006DAF074009006DBF0800C74F0
:103E3900009000ADF074199006DAF09000C6E0B475
:103E49000214741A9000AEF074009006DEF074004B
:103E59009006DFF0800C74009000AEF0741A9006A2
:103E6900DEF09000E4E0D394014014741B90011734
:103E7900F074009006E2F074009006E3F0800C7490
:103E890000900117F0741B9006E2F09000F2E0B484
:103E99000114741C900118F074009006E6F0740087
:103EA9009006E7F0800C7400900118F0741C9006DD
:103EB900E6F09000D4E0B402069000F2E0600280DF
:103EC9001A74059006EAF074069006EEF0740790ED
:103ED90006F2F074089006F6F0803074009006EA55
:103EE900F074009006EBF074009006EEF074009008
:103EF90006EFF074009006F2F074009006F3F07487
:103F0900009006F6F074009006F7F0D22C9000C6E7
:103F1900E0900087F09000F2E0900088F09000E4D3
:103F2900E0900089F09000D4E090008AF090009928
:103F3900E090008BF0900099E090006FF09000D431
:103F4900E0900073F09000F2E0900074F09000C6E9
:103F5900E0900075F09000E4E0900076F09000FCAD
:103F6900E0B40117900027740FF0A374FFF09000DC
:103F790029E4F0A3F074029000FCF09000FCE0B496
:103F89000341900029E0FEA3E0FF900027E0FCA395
:103F9900E0FD126FE87410126F9C7408120039EF7B
:103FA900900080F0EF700674FF900080F07400902C
:103FB90000FCF0900028E0900081F0900027E0904C
:103FC9000082F090008DE090004BF090004BE024CF
:103FD9000F90004CF090004BE0241E90004DF090A3
:103FE900004BE0242D90004EF090004CE0D3943C1F
:103FF900400B90004CE0C3943C90004CF090004D75
:10400900E0D3943C400B90004DE0C3943C90004DAC
:10401900F090004EE0D3943C400B90004EE0C394E6
:104029003C90004EF0900053E4F090004BE0643B6C
:10403900600790004BE0B43C2090004BE0B43B0695
:104049007402900053F090004BE0B43C069000538A
:104059007401F090004B7401F0900054E4F090006A
:104069004CE0643B600790004CE0B43C2090004C6D
:10407900E0B43B067402900054F090004CE0B43C6C
:10408900069000547401F090004C7401F0900055B2
:10409900E4F090004DE0643B600790004DE0B43CD3
:1040A9002090004DE0B43B067402900055F090005A
:1040B9004DE0B43C069000557401F090004D740138
:1040C900F090004EE0643B600790004EE0B43C2065
:1040D90090004EE0B43B067402900056F090004EFA
:1040E900E0B43C069000567401F090004E7401F063
:1040F90090008DE0FE9000F0E02E900058F09000C6
:1041090058E0641E6007900058E0B43C06900058DF
:10411900E004F0900058E0641D6007900058E0B496
:104129003B06900058E014F0900058E0D3943C40CE
:104139000B900058E0C3943C900058F0900058E070
:10414900D3941E400D900058E0C3941E900059F07E
:10415900800A900058E0241E900059F075511E9075
:1041690000D3E090004FF090004FE075F00F84AF5E
:10417900F07E00EF4E700690004FE004F090004F83
:10418900E00475F00F84AFF07E00EF4E70069000EA
:104199004FE014F090004FE0B4790690004F74019D
:1041A900F090004FE0D3943C400F90004FE0C3944F
:1041B9003C90004FF0D2268002C22690004FE024A6
:1041C9000F900050F090004FE0241E900051F090A5
:1041D900004FE0242D900052F0900050E0D3943C21
:1041E900400B900050E0C3943C900050F090005177
:1041F900E0D3943C400B900051E0C3943C900051B3
:10420900F0900052E0D3943C400B900052E0C394EC
:104219003C900052F022C293C294C291C292C287CA
:10422900C290E5B554EFF5B5E5B554DFF5B5C296DD
:10423900C295C2A0C297C2A2C2A1E5B554BFF5B545
:10424900E5B5547FF5B5E5B554FBF5B5C212755E14
:10425900469000D6E07005756D028003756D037593
:10426900550075540090001074FFF0A374DCF0C27F
:1042790019C21BC21DC21F74C890003BF074C890BC
:10428900003FF074C8900043F074C8900047F0757F
:104299005300755200C20D754600E56FB4090375E8
:1042A9006F0075630090001DE4F0A3F0757010C2F3
:1042B90015C216C217C2189007C6E0FEA3E0FF7424
:1042C90003126F9C74011200399007C4EEF0A3EF3A
:1042D900F0C202755700755600900014E4F0A3F07F
:1042E900C22E755900755800900098E075F032A4F7
:1042F900FDACF0900025ECF0A3EDF0C23EA232B384
:104309009205A233B39206A234B39207A235B392AF
:1043190008A236B39209A237B3920AA238B3920B14
:10432900A239B3920C2285F97385FA747E017F0054
:10433900E574126F9CE5732FFF50010E8E5A8F5B47
:10434900AC5CAD5DEF2DFDEE3CFC8C5C8D5D123AF5
:10435900E9123AF4123AFF123B0A9000D4E0B4038E
:104369002C75A71085F97385FA747E017F00E574B1
:10437900126F9CE5732FFF50010E8E5A8F5B123B13
:1043890015123B20123B2B123B3A75A7002275A749
:104399001085F97385FA747E017F00E574126F9CAC
:1043A900E5732FFF50010E8E5A8F5B7E017F769049
:1043B9000111E0126F9CAC5AAD5BED2FFFEC3EFE94
:1043C9008E5C8F5DE55DF5FDE55CF5FE900084E4AE
:1043D900F075A700741290005BF02285F97385FAD5
:1043E900747E017F00E574126F9CE5732FFF500105
:1043F9000E8E5A8F5B9007C6E0FCA3E0FDEF2DFD02
:10440900EE3CFC8C5C8D5DE55DF5FDE55CF5FE2221
:104419000564229000D4E0640360079000F2E0B4E0
:10442900021EA2D8B34002C293A2D9B34002C294D9
:10443900A2DAB34002C291A2DBB34002C292804425
:10444900A2D8B3400AC2939000F2E06002C287A2E8
:10445900D9B3400AC2949000F2E06002C290A2DA95
:10446900B3400EC2919000F2E06006E5B554EFF555
:10447900B5A2DBB3400EC2929000F2E06006E5B54A
:1044890054DFF5B5A2DCB34008C296C295C2A0C2FA
:104499009775D8402285A77275A7109000D4E0645B
:1044A9000360079000F2E0B40224A2D8B34002C22C
:1044B90087A2D9B34002C290A2DAB34006E5B55447
:1044C900EFF5B5A2DBB34006E5B554DFF5B5A2DCDF
:1044D900B340089000E0E0900084F075D840857200
:1044E900A722900047E4936406600280FE74C89096
:1044F90007CCF8E4F0E8A3F075B50075840175A759
:104509000075FFA0900057E4F075C91075A70F75E5
:10451900A1C775A70075D90075CE0C75A70F75F1E0
:10452900FE75F2FF75F30775F47875A4BA75A5FFE2
:1045390075A60775AE0075AFFF75D48175D5FF7582
:10454900D6FF75D7FF75A70075A20175A14775F844
:104559000975D80075D90475DA0975DB0975DC099F
:1045690075DD0975DE0975D84075A71075D8007510
:10457900D90475DA0975DB0975DC0975DD0975DE9C
:104589000975D84075A70075E60875E71075BC016F
:1045990075BE0475BD6C75BE0775BDA075BE087581
:1045A900BD0175BC0075BB1875BC2075BA0875E8E6
:1045B9008075D11375A70F75E10575E20075C740C0
:1045C90012421F759700759780740A126F7C759750
:1045D900C0E5975420700280F8758F0275A700D244
:1045E900AF75980075A90C75A70F75AB4375ADFB31
:1045F90075AC1E75A71075C91875CA0075CB0075FD
:10460900C80475A700758912758E04758C00758AA2
:1046190000C2A9D28C758D00758B00D2ABD28E7574
:10462900EF0675D944C2997509C87508001200E9E1
:1046390075B5001204E974639007CCF8E4F0E8A3B7
:10464900F012037574C89007CCF8E4F0E8A3F0758C
:1046590009647508001200E990006FE0900099F074
:10466900900099E0D39403400C7400900099F07481
:104679000090006FF0C223900099E09067DEF8285F
:1046890028738028A2B44002D223802075A70F7511
:10469900F30F75A700A2A34002D223800F75A70FBD
:0C46A90075F31775A700A2A44002D223ED
:0C67DE0002468B02468D0246950246A63C
:1046B500A223B3405E757308E573D3940E501FE5CE
:1046C500739007CCF8E4F0E8A3F01202447509648E
:1046D5007508001200E97873740126F650DA740241
:1046E5009000D5F090006FE0900099F0900099E06F
:1046F5009067EAF8282873801674009000FFF08010
:0F4705000E74009000E4F0800674009000F1F054
:0C67EA000246FC0246FE02470602470E73
:10471400D222805C757301E573D39407501FE5734F
:104724009007CCF8E4F0E8A3F0120244750964752C
:1047340008001200E97873740126F650DA740190C7
:1047440000D5F090006FE0900099F0900099E0900F
:1047540067F6F8282873801674009000FFF0800E26
:0E47640074009000E4F0800674009000F1F004
:0C67F60002475A02475C02476402476CED
:10477200C22290006EE090012AF090006FE090005B
:1047820099F0900070E09000B9F0900071E0900014
:10479200E2F0900072E090008EF0900073E09000E2
:1047A200D4F0900074E09000F2F0900075E0900078
:1047B200C6F0900076E09000E4F0900077E090017F
:1047C20014F0900078E0900178F0900079E0900188
:1047D20079F090007AE090017AF0900178E0700C24
:1047E200900179E0700690017AE060028004C22DA7
:1047F2008002D22D9000DFE07006740A9000DFF094
:104802009000C0E0700674E39000C0F09000C6E033
:1048120004900087F09000C7E09000F9F0123BE0AE
:10482200E5B54401F5B5740690005DF074019000A1
:104832005EF07403900060F07405900061F0741FE4
:10484200900062F07405900063F090005FE0B404A1
:10485200067404900063F07401900064F074009098
:104862000069F0740090006CF074FF90006DF074B9
:1048720036900163F07430900164F0742D900165FC
:10488200F07432900166F07420900167F0743890F1
:104892000168F07443900169F0747990016AF074D0
:1048A2006C90016BF0742090016CF0742090016D9B
:1048B200F0742090016EF0742090016FF0742090DB
:1048C2000170F07420900171F09000FBE090008084
:1048D200F09000B2E0900081F09000B3E09000828E
:1048E200F0A2B6B3920EA2B3B3920FA2A4B39229CE
:1048F200A2B4B3922AA2A3B3922B90007CE4F075E7
:104902006F00743A90078CF074FD90078DF0900060
:104912007DE4F09007C6E0FEA3E0FF7403126F9CF3
:1049220074011200399007C4EEF0A3EFF0756E0126
:1049320090005BE4F0C228756300C213D214C20275
:10494200757100C230D203C231D204C232D205C262
:1049520033D206C234D207C235D208C236D209C215
:1049620037D20AC238D20BC239D20CC224C225C2F3
:1049720026C227C22C12009E755F00756B007561FE
:1049820000756532756600756700756800756900A7
:10499200756A0090001DE4F0A3F0756C00D2B2D2EB
:1049A200A4D2B0D2B1D2A3D2A7D2A6D2A5D2B79066
:1049B2000098E0D394FA400674FA900098F07E01D1
:1049C2007F00900082E0126F9C900081E02FFF50E8
:1049D200010E900027EEF0A3EFF0EFD394FFEE94D8
:1049E2000F4007900027E4F0A3F0900080E07006EB
:1049F20074FF900080F09000D5E0D39402400674DA
:104A0200019000D5F09000D6E07005756D0280032C
:104A1200756D039000D7E0D39401400674009000B6
:104A2200D7F09000DDE0C3940A5006740A9000DDCE
:104A3200F09000E7E0700674019000E7F09000E764
:104A4200E0B4FF0674FE9000E7F09000EEE0D3942D
:104A5200FE400674FE9000EEF0900114E0D3940242
:104A620040067401900114F090012AE0D3940140B1
:104A720006740190012AF074019000F4F074019020
:104A820000F5F074009000FCF0740090011CF074CA
:104A9200299006D2F0742A9006D6F0D29C9000C7D4
:104AA200E0D39404400674049000C7F0E570D394F8
:104AB2001040037570109006D3E0D3940C40067436
:104AC200009006D3F09006D7E0D3940C4006740011
:104AD2009006D7F09006DBE0D3940C400674009069
:104AE20006DBF09006DFE0D3940C400674009006DB
:104AF200DFF09006E3E0D3940C400674009006E3E6
:104B0200F09006E7E0D3940C400674009006E7F0BC
:104B12009006EBE0D3940C400674009006EBF09004
:104B220006EFE0D3940C400674009006EFF0900676
:104B3200F3E0D3940C400674009006F3F09006F76D
:104B4200E0D3940C400674009006F7F0D2EC75CFD7
:104B520001A298B34005C298120646E54D6006A22E
:104B620099B3B340028005C299120C57E54E640115
:104B72006005E54EB4040280D5C28E7E107F00E54A
:104B820064126F9CE58D75F010A4FDACF0EF2DFD65
:104B9200EE3CFCE58B75F01084FF7E00ED2FFFEC00
:104BA2003EFE8E548F55D28E9000B9E0600990007F
:104BB200B9E0C3943D4002805C90001F126FAA903E
:104BC200001FE0FEA3E0FF900021E0FCA3E0FDEF68
:104BD200B50542EEB5043EB221A20DB3401975E708
:104BE20000A221B34008E5B54404F5B58006E5B559
:104BF20054FBF5B575E710900021E0FEA3E0FF90AD
:104C02000023E0FCA3E0FDEF2DFDEE3CFC90002133
:104C1200ECF0A3EDF09000C6E060099000C6E0C39E
:104C220094034002806F122D96A20DB3500990009A
:104C32007CE0C3942B400280069000B0E0F545E58D
:104C42004575F005A4FFAEF09007CEEEF0A3EFF0AD
:104C520090009DE0C395614007E55FC395605007F2
:104C62009007CEE4F0A3F0AE2EAF2F9007CEE0FC7B
:104C7200A3E0FDEFD39DEE9C4004C2A1800B900007
:104C82007CE0C394415002D2A19000C6E0B4020578
:104C9200A2A1B392A29000C6E0B4031C122EB1AE40
:104CA2002EAF2F9007CEE0FCA3E0FDEFD39DEE9C4C
:104CB2004004D2A18002C2A19000A1E06009A2B387
:104CC200300F01B3B340028039A2B3300F01B340B9
:104CD20031A2B3301101B3401C9000D4E0B40306FA
:104CE200A224B3B340028006740490005BF0D22485
:104CF200A211B3920FA211B330B301B34004A211B7
:104D0200920FA2B6300E01B350030253DAA2B630AC
:104D12000E01B350030253DAA2B6301001B35003AE
:104D22000251DC756E009000B9E0B43D1975E700E0
:104D3200A210B34008E5B554FBF5B58006E5B544CD
:104D420004F5B575E710055EA212B3B35013AE5465
:104D5200AF55900010E0FCA3E0FDEDC39FEC9E4038
:104D620003024EB9E56DB4032EA22EB34022E55ED6
:104D7200B43B03756D01E55EC3943B500690005B46
:104D82007401F0E55ED3943B4006740290005BF040
:104D9200755E01D22E805EE56DB40206756D0175F9
:104DA2005E3BE55EB43B05755E01804990005BE0C9
:104DB2007034E55EC3943B500690005B7401F0E5ED
:104DC2005ED3943B4006740290005BF0E55EC394B0
:104DD2003B5002D228E55ED3943B4002D228C296D1
:104DE200C295C2A0C2979000D6E0B4010512421F3C
:104DF2008003755E01AE56AF57AC54AD55EF2DFD35
:104E0200EE3CFC74028C068D071200398E568F57C9
:104E12009000B9E060099000B9E0C3943D4002807F
:104E22004990001FE0FEA3E0FF9000B9E08E048FDE
:104E320005FF126F8C74018C068D071200399000E9
:104E420023EEF0A3EFF0900023E0F8A3E09000211E
:104E5200C8F0A3C8F090001FE4F0A3F0C22175E7E8
:104E620000E5B554FBF5B575E710A2B4B34002C234
:104E72002AA2A4B34002C229A2A3B34002C22BA217
:104E820028B34002C228A224B34006A2269225805B
:104E920002B2259000A1E06012E56D700EA224B36B
:104EA2005009A225302601B3B34002800674059052
:104EB200005BF0C224803AAE56AF57AC54AD55EF0A
:104EC2002DFDEE3CFC74018C068D071200398E56C6
:104ED2008F57E56DC39402500DAC54AD5574B8C3F1
:104EE2009D740B9C4002800912421F740690005B65
:104EF200F0E55EB43B12740390005BF0D2289000A0
:104F0200D6E0B4010312421FAE58AF59AC54AD55AE
:104F1200EF2DFDEE3CFC8C588D59AE54AF55EFD3BE
:104F22009DEE9C4011900017E0FAA3E0FBEBC394C6
:104F3200E8EA940340028006900017126FAA9000DC
:104F420014E0FEA3E0FFAC54AD55EF2DFDEE3CFCAA
:104F5200900014ECF0A3EDF09000D6E0B40118AE8E
:104F620054AF557405126F9C7401120039900010F1
:104F7200EEF0A3EFF08011AE54AF557402126F9CA5
:104F8200900010EEF0A3EFF0C28E758D00758B00CD
:104F9200756400755501755400D28EE55E240E7558
:104FA200F00F84AFF07E00EF4E7075900014E0F8C1
:104FB200A3E0900012C8F0A3C8F0900012E0FEA394
:104FC200E0FFEF4E600B7C7A7DF8126E8A8E528F74
:104FD20053900014E4F0A3F0AE52AF537428BE0015
:104FE200039F5010E5632FFF50010E740112003928
:104FF2008E528F538553639000DDE0A852B8000DA6
:10500200D395534008E55390005AF080099000DD93
:10501200E01490005AF0E56D600675530075520079
:105022009000D4E0B4030890004FE0655E60028017
:105032000BA225B34004D2278002B227E55E640B9F
:105042006005E55EB429099000C6E060031223D230
:10505200900058E0655E6007900059E0B55E037508
:105062006F00A213B35006A212B3B340030251174A
:10507200900092E0B40173900114E0B40214120E95
:1050820026900085E075F0BEA4FFAEF08E5C8F5DC9
:105092008056E56775F00A84FF7E0090058C126FDA
:1050A200C3E0F55B755A00AE5AAF5B9000B7E012F1
:1050B2006F9C74648E048F05FF126F8C8C5C8D5D07
:1050C200E55D900016F0AE5AAF5B900090E0126F73
:1050D2009C74648E048F05FF126F8C74BE8C068DD7
:1050E20007126F9C8E5C8F5D8017900090E075F0C8
:1050F200BEA4FFAEF08E5C8F5D9000B7E09000160C
:10510200F0E561C394CC5006E55D455C7002800316
:1051120012432FD213E56DB40106E55E64116002FD
:10512200800975700190005C7401F0E56D60030206
:1051320051D79000D9E0600D900084E0A852B800E9
:10514200069553400280489000D9E0B402279000AF
:105152004BE0655E601790004CE0655E600F90006A
:105162004DE0655E600790004EE0B55E037570032A
:10517200756C00800CC200756C0090001DE4F0A3F9
:10518200F0900084E06006740990005BF080469025
:10519200004BE0B55E0B75700190005C7401F0800D
:1051A2003490004CE0B55E0B757001740290005CA7
:1051B200F0802290004DE0B55E0B75700174039093
:1051C200005CF0801090004EE0B55E0975700174CD
:1051D2000490005CF0A210B3920EA210B330B6019C
:1051E200B350030253DA756E019000B9E0B43D1971
:1051F20075E700A210B34008E5B54404F5B5800692
:10520200E5B554FBF5B575E71075E700E5B5440162
:10521200F5B575E710742B90007CF0A210920EE5A4
:105222005ED3944A4014D212E55ED39485400B7447
:105232000490005BF0D228755E469000E1E0B40174
:1052420007E56AC394144002800912421F74139046
:10525200005BF0A230300301B3501D75E700A230AD
:10526200B34008E5B54408F5B58006E5B554F7F551
:10527200B575E710A2309203A231300401B3501D7C
:1052820075E700A231B34008E5B54402F5B58006E2
:10529200E5B554FDF5B575E710A2319204A232309E
:1052A2000501B3500FA232B34004D2A28002C2A2BF
:1052B200A2329205A233300601B3500FA233B3409B
:1052C20004D2A18002C2A1A2339206A23430070105
:1052D200B3501D75E700A234B34008E5B54440F56C
:1052E200B58006E5B554BFF5B575E710A23492074F
:1052F200A235300801B3501D75E700A235B340084E
:10530200E5B54480F5B58006E5B5547FF5B575E79A
:1053120010A2359208A236300901B3500FA236B35B
:105322004004D2878002C287A2369209A237300A8D
:1053320001B3500FA237B34004D2908002C290A2B0
:1053420037920AA238300B01B3501D75E700A2381C
:10535200B34008E5B54410F5B58006E5B554EFF560
:10536200B5A238920B75E710A239300C01B3501D6B
:1053720075E700A239B34008E5B54420F5B58006CB
:10538200E5B554DFF5B5A239920C75E710E56AC3AD
:1053920094415009740E90005BF012421F9000631A
:1053A200E0FE90005FE004C39E400990005FE0D3FE
:1053B2009408400974FB90005BF012421F90006851
:1053C200E06015900068E0FE900062E06E60097493
:1053D200FE90005BF012421FA228B34008C296C2A0
:1053E20095C2A0C297900111E0600CAE52AF537407
:1053F20014BE00059F40028048900099E090680228
:10540200F8282873803BA2B4B35005A22AB3400205
:105412008005124397D22A8028A2A3B35005A22B5B
:10542200B340028005124397D22B8015A2A4B35039
:1054320005A229B340028005124397D22980028037
:015442000069
:1068020002540602540802541B02542E025441023E
:026812005443ED
:10544300A215B3B3500890004FE0655E60030255A8
:1054530018A201B35006A200B3B340030255109043
:1054630000D4E0B4036EA20DB34038A227B34008C2
:10547300123A8C123AE98009123AB9123B1575A710
:10548300009000F2E0B4011975E700A202B34008EE
:10549300E5B54480F5B58006E5B5547FF5B575E708
:1054A30010802F123A8C123AE9123AB9123B157551
:1054B300A7009000F2E0B4011975E700A202B3401F
:1054C30008E5B54480F5B58006E5B5547FF5B575B7
:1054D300E71080399000F2E0C39402500F123A8C27
:1054E300123AE9A202B34002D2878021123A8C1207
:1054F3003AE9123AB9AE5AAF5BAC2CAD2DEF2DFDA4
:10550300EE3CFC8C5C8D5D123B1575A700C215D279
:1055130016D217D218A216B3B35008900050E06504
:105523005E60030255EDA201B35006A200B3B3407F
:10553300030255E59000D4E0B4036EA20DB34038E6
:10554300A227B34008123A8C123AF48009123AB9EE
:10555300123B2075A7009000F2E0B4011975E70033
:10556300A202B34008E5B54480F5B58006E5B5541D
:105573007FF5B575E710802F123A8C123AF4123A80
:10558300B9123B2075A7009000F2E0B4011975E74A
:1055930000A202B34008E5B54480F5B58006E5B541
:1055A300547FF5B575E71080399000F2E0C394029B
:1055B300500F123A8C123AF4A202B34002D29080F6
:1055C30021123A8C123AF4123AB9AE5AAF5BAC2CB0
:1055D300AD2DEF2DFDEE3CFC8C5C8D5D123B2075FB
:1055E300A700D215C216D217D218A217B3B3500808
:1055F300900051E0655E60030256C6A201B35006F7
:10560300A200B3B340030256BE9000D4E0B4036ECD
:10561300A20DB34038A227B34008123A8C123AFFC6
:105623008009123AB9123B2B75A7009000F2E0B43F
:10563300011975E700A202B34008E5B54480F5B54A
:105643008006E5B5547FF5B575E710802F123A8CC7
:10565300123AFF123AB9123B2B75A7009000F2E001
:10566300B4011975E700A202B34008E5B54480F51B
:10567300B58006E5B5547FF5B575E710803D90001C
:10568300F2E0C394025013123A8C123AFFA202B30F
:105693004006E5B54410F5B58021123A8C123AFF65
:1056A300123AB9AE5AAF5BAC2CAD2DEF2DFDEE3CEB
:1056B300FC8C5C8D5D123B2B75A700D215D216C2F4
:1056C30017D218A218B3B35008900052E0655E6079
:1056D3000302579FA201B35006A200B3B3400302D3
:1056E30057979000D4E0B4036EA20DB34038A227BD
:1056F300B34008123A8C123B0A8009123AB9123BA2
:105703003A75A7009000F2E0B4011975E700A20210
:10571300B34008E5B54480F5B58006E5B5547FF59B
:10572300B575E710802F123A8C123B0A123AB91260
:105733003B3A75A7009000F2E0B4011975E700A2A7
:1057430002B34008E5B54480F5B58006E5B5547F5E
:10575300F5B575E710803D9000F2E0C39402501355
:10576300123A8C123B0AA202B34006E5B54420F577
:10577300B58021123A8C123B0A123AB9AE5AAF5B8A
:10578300AC2CAD2DEF2DFDEE3CFC8C5C8D5D123B06
:105793003A75A700D215D216D217C218E5709068D1
:0C57A30014F8282873025DBA9000C7E0DB
:066814000257A80257AB79
:1057AF00906847F8282873121EAE8012121EAE8022
:0E57BF000D121F388008121FE48003121FE431
:0F6847000257B60257BB0257C00257C50257CAC5
:1057CD00757002025DBA122110122227A23EB3405B
:1057DD00229000BBE0F56C90008CE0256CFE9000F3
:1057ED005AE075F01E84FC7F00EE2CF53674109097
:1057FD00005BF09007C4E0FEA3E0FF740A126F9CFB
:10580D00900012E0FCA3E0FD74098F02FF126F8C73
:10581D008D078C038E048A058B06126E8A9007C83D
:10582D00EEF0A3EFF09000E2E0B40108743CBE008E
:10583D00059F4002800D743C9007C8F8E4F0E8A382
:10584D00F0801B9007C8E0FEA3E0FF74F0BE0003DC
:10585D009F500B74F09007C8F8E4F0E8A3F0E5361C
:10586D0070037536019007C8E0FEA3E0FFE5362F03
:10587D00FF50010E9007C8EEF0A3EFF07570039086
:03588D00005CE0DC
:03681A000257D34F
:10589000906856F82828738022A23F400375700A4A
:1058A0008019A23F400375700B8010A23F40037522
:0B58B000700C8007A23F400375700DD4
:0F6856000258970258990258A20258AB0258B440
:1058BB00025DBA9006D3E060031224EA900112E075
:1058CB00B40114900113E0A852B80004955350078B
:1058DB00E55FC3956040028009741590005BF00290
:1058EB00596E9000C7E0D39402403F90009BE02498
:1058FB0003A852B800049553500990009DE0D3952E
:10590B006150028008D201740890005BF090009BFC
:10591B00E0A852B80005D39553500B90009DE0249E
:10592B0003C395615002C201803990009BE02403B0
:10593B00A852B8000495535007E55FC39560400229
:10594B008008D201740890005BF090009BE0A85295
:10595B00B80005D395535009E560240FC3955F50EC
:10596B0002C2019000E1E07007E56AC394144002A3
:10597B008002D201A2014005757004800A75701077
:10598B0090001DE4F0A3F0A20DB34029E56775F07C
:10599B000A84FF7E0090058C126FC3E0C39469509C
:1059AB0005122407800F9007C6E0F8A3E09007C408
:0C59BB00C8F0A3C8F0025DBA9000C7E07D
:06681D000258BE0259C33F
:1059C700906865F8282873120F108012120F108044
:0E59D7000D1210BE80081211708003121170A4
:0F6865000259CE0259D30259D80259DD0259E225
:1059E5009006D7E060031225C6757005025DBA12F0
:1059F50012B07570069006DBE060031226B69006BD
:105A0500DFE06003122792025DBA900016E060069F
:105A1500A20DB3B34002801D900016E02529FFAE0C
:105A25002850010E8E288F29E55ED3940F500690DD
:105A35000016E014F01214F67570079006E3E060A6
:105A45000312286E9006E7E0600312294A025DBA48
:105A5500900114E0B40203120E9E1218F575700839
:105A65009006EBE06003122A269006EFE060031231
:105A75002B02025DBA121CB1A215B35005A216B3D2
:105A850040028008D215D216D217D2187570109020
:105A950006F3E06003122BDE9006F7E06003122C9C
:105AA500BA025DBA025DBA90003DE0C39446500863
:105AB500C296744690003DF0900053E0B4011DE598
:105AC500362406F5369007C8E0FEA3E0FF74062FDE
:105AD500FF50010E9007C8EEF0A3EFF0900053E0E1
:105AE500B4021DE536240CF5369007C8E0FEA3E0A8
:105AF500FF740C2FFF50010E9007C8EEF0A3EFF0D6
:105B050085365B755A0090004BE0F573123B49E50D
:105B15005D90003DF0900008E55AF0A3E55BF0E5E7
:105B25007390003EF0C21A9007C8E0F55AA3E0F55D
:105B35005B90004BE0F573123B49E55D90003BF04F
:105B4500900000E55AF0A3E55BF0E57390003CF0AA
:105B5500C219E56DB4010575700B800375700302FC
:105B65005DBA900041E0C3944650139000E2E0B462
:105B75000104C2968002C2957446900041F09000DF
:105B850054E0B4011DE5362406F5369007C8E0FE5D
:105B9500A3E0FF74062FFF50010E9007C8EEF0A397
:105BA500EFF0900054E0B4021DE536240CF5369074
:105BB50007C8E0FEA3E0FF740C2FFF50010E90070D
:105BC500C8EEF0A3EFF085365B755A0090004CE007
:105BD500F573123B49E55D900041F090000AE55AE6
:105BE500F0A3E55BF0E573900042F0C21C9007C896
:105BF500E0F55AA3E0F55B90004CE0F573123B49E4
:105C0500E55D90003FF0900002E55AF0A3E55BF0FA
:105C1500E573900040F0C21BE56DB4010575700C8D
:105C25008003757003025DBA900045E0C394465049
:105C3500139000E2E0B40104C2968002C2A074464B
:105C4500900045F0900055E0B4011DE5362406F5B9
:105C5500369007C8E0FEA3E0FF74062FFF50010E43
:105C65009007C8EEF0A3EFF0900055E0B4021DE5F3
:105C750036240CF5369007C8E0FEA3E0FF740C2F20
:105C8500FF50010E9007C8EEF0A3EFF085365B7567
:105C95005A0090004DE0F573123B49E55D900045D3
:105CA500F090000CE55AF0A3E55BF0E57390004633
:105CB500F0C21E9007C8E0F55AA3E0F55B90004DD1
:105CC500E0F573123B49E55D900043F0900004E573
:105CD5005AF0A3E55BF0E573900044F0C21DE56D55
:105CE500B4010575700D8003757003025DBA9000EF
:105CF50049E0C3944650139000E2E0B40104C29613
:105D05008002C2977446900049F0900056E0B401B5
:105D15001DE5362406F5369007C8E0FEA3E0FF74BE
:105D2500062FFF50010E9007C8EEF0A3EFF090008C
:105D350056E0B4021DE536240CF5369007C8E0FEA2
:105D4500A3E0FF740C2FFF50010E9007C8EEF0A3DF
:105D5500EFF085365B755A0090004EE0F573123B07
:105D650049E55D900049F090000EE55AF0A3E55B2A
:105D7500F0E57390004AF0C2209007C8E0F55AA3F9
:105D8500E0F55B90004EE0F573123B49E55D900050
:105D950047F0900006E55AF0A3E55BF0E573900047
:105DA50048F0C21FE56DB40103756D007570038081
:055DB5000480028000E3
:106823000259F4025A0F025A55025A7A025AA9021D
:106833005AAC025B67025C2D025CF3025DB6025D3B
:04684300B8025DBA80
:105DBA0090003BE0B55E028003025E5CA21940726D
:105DCA00900000E0FEA3E0FFEF4E6021AE56AF5711
:105DDA00900000E0FCA3E0FD12000374068E048F1D
:105DEA0005FF126F8C900000ECF0A3EDF090003CE0
:105DFA00E0601A900000E0FEA3E0FFAC56AD57EF5A
:105E0A002DFDEE3CFC900000ECF0A3EDF090003C80
:105E1A00E0D39401401A900000E0FEA3E0FFAC56E4
:105E2A00AD57EF2DFDEE3CFC900000ECF0A3EDF039
:105E3A00D219AE54AF55900000E0FCA3E0FDEFC3C9
:105E4A009DEE9C400D1243E4D296C21974C890008C
:105E5A003BF0A219B3B3500790003BE0B55E028055
:105E6A000D1243E4D29674C890003BF0C219900018
:105E7A003DE0B55E028003025F17A21A40729000ED
:105E8A0008E0FEA3E0FFEF4E6021AE56AF57900048
:105E9A0008E0FCA3E0FD12000374068E048F05FFE0
:105EAA00126F8C900008ECF0A3EDF090003EE060D9
:105EBA001A900008E0FEA3E0FFAC56AD57EF2DFDA7
:105ECA00EE3CFC900008ECF0A3EDF090003EE0D32D
:105EDA009401401A900008E0FEA3E0FFAC56AD57CB
:105EEA00EF2DFDEE3CFC900008ECF0A3EDF0D21A89
:105EFA00AE54AF55900008E0FCA3E0FDEFC39DEE61
:105F0A009C400AC296744690003DF0C21AA21AB387
:105F1A00B3500790003DE0B55E02800AC29674460F
:105F2A0090003DF0C21A90003FE0B55E0280030285
:105F3A005FDDA21B4072900002E0FEA3E0FFEF4E7D
:105F4A006021AE56AF57900002E0FCA3E0FD1200BC
:105F5A000374068E048F05FF126F8C900002ECF01A
:105F6A00A3EDF0900040E0601A900002E0FEA3E08A
:105F7A00FFAC56AD57EF2DFDEE3CFC900002ECF065
:105F8A00A3EDF0900040E0D39401401A900002E0A3
:105F9A00FEA3E0FFAC56AD57EF2DFDEE3CFC9000A2
:105FAA0002ECF0A3EDF0D21BAE54AF55900002E024
:105FBA00FCA3E0FDEFC39DEE9C40181243E4900061
:105FCA00E2E0B40104D2968002D295C21B74C89052
:105FDA00003FF0A21BB3B3500790003FE0B55E024A
:105FEA0080181243E49000E2E0B40104D2968002E1
:105FFA00D29574C890003FF0C21B900041E0B55E94
:10600A000280030260AEA21C407290000AE0FEA366
:10601A00E0FFEF4E6021AE56AF5790000AE0FCA3B6
:10602A00E0FD12000374068E048F05FF126F8C9038
:10603A00000AECF0A3EDF0900042E0601A90000A2A
:10604A00E0FEA3E0FFAC56AD57EF2DFDEE3CFC9011
:10605A00000AECF0A3EDF0900042E0D39401401A5C
:10606A0090000AE0FEA3E0FFAC56AD57EF2DFDEE1F
:10607A003CFC90000AECF0A3EDF0D21CAE54AF55F4
:10608A0090000AE0FCA3E0FDEFC39DEE9C40159052
:10609A0000E2E0B40104C2968002C2957446900000
:1060AA0041F0C21CA21CB3B35007900041E0B55E98
:1060BA000280159000E2E0B40104C2968002C29503
:1060CA007446900041F0C21C900043E0B55E028025
:1060DA000302617FA21D4072900004E0FEA3E0FF6C
:1060EA00EF4E6021AE56AF57900004E0FCA3E0FDEE
:1060FA0012000374068E048F05FF126F8C90000441
:10610A00ECF0A3EDF0900044E0601A900004E0FE89
:10611A00A3E0FFAC56AD57EF2DFDEE3CFC9000041A
:10612A00ECF0A3EDF0900044E0D39401401A900003
:10613A0004E0FEA3E0FFAC56AD57EF2DFDEE3CFCAC
:10614A00900004ECF0A3EDF0D21DAE54AF559000D0
:10615A0004E0FCA3E0FDEFC39DEE9C40181243E46B
:10616A009000E2E0B40104D2968002D2A0C21D746B
:10617A00C8900043F0A21DB3B35007900043E0B5A6
:10618A005E0280181243E49000E2E0B40104D29661
:10619A008002D2A074C8900043F0C21D900045E06E
:1061AA00B55E028003026250A21E407290000CE0AB
:1061BA00FEA3E0FFEF4E6021AE56AF5790000CE011
:1061CA00FCA3E0FD12000374068E048F05FF126F14
:1061DA008C90000CECF0A3EDF0900046E0601A9071
:1061EA00000CE0FEA3E0FFAC56AD57EF2DFDEE3CF0
:1061FA00FC90000CECF0A3EDF0900046E0D3940183
:10620A00401A90000CE0FEA3E0FFAC56AD57EF2D0C
:10621A00FDEE3CFC90000CECF0A3EDF0D21EAE5467
:10622A00AF5590000CE0FCA3E0FDEFC39DEE9C404F
:10623A00159000E2E0B40104C2968002C2A074463E
:10624A00900045F0C21EA21EB3B35007900045E06D
:10625A00B55E0280159000E2E0B40104C2968002A5
:10626A00C2A07446900045F0C21E900047E0B55E99
:10627A00028003026321A21F4072900006E0FEA37F
:10628A00E0FFEF4E6021AE56AF57900006E0FCA348
:10629A00E0FD12000374068E048F05FF126F8C90C6
:1062AA000006ECF0A3EDF0900048E0601A900006BA
:1062BA00E0FEA3E0FFAC56AD57EF2DFDEE3CFC909F
:1062CA000006ECF0A3EDF0900048E0D39401401AE8
:1062DA00900006E0FEA3E0FFAC56AD57EF2DFDEEB1
:1062EA003CFC900006ECF0A3EDF0D21FAE54AF5583
:1062FA00900006E0FCA3E0FDEFC39DEE9C4018125F
:10630A0043E49000E2E0B40104D2968002D297C23C
:10631A001F74C8900047F0A21FB3B35007900047FC
:10632A00E0B55E0280181243E49000E2E0B4010492
:10633A00D2968002D29774C8900047F0C21F90008C
:10634A0049E0B55E0280030263F2A2204072900027
:10635A000EE0FEA3E0FFEF4E6021AE56AF5790006D
:10636A000EE0FCA3E0FD12000374068E048F05FF05
:10637A00126F8C90000EECF0A3EDF090004AE060F2
:10638A001A90000EE0FEA3E0FFAC56AD57EF2DFDCC
:10639A00EE3CFC90000EECF0A3EDF090004AE0D346
:1063AA009401401A90000EE0FEA3E0FFAC56AD57F0
:1063BA00EF2DFDEE3CFC90000EECF0A3EDF0D220A8
:1063CA00AE54AF5590000EE0FCA3E0FDEFC39DEE86
:1063DA009C40159000E2E0B40104C2968002C29784
:1063EA007446900049F0C220A220B3B3500790002F
:1063FA0049E0B55E0280159000E2E0B40104C2965D
:10640A008002C2977446900049F0C2209000E4E0EE
:10641A00B40202800302654790007EE0D39566507D
:10642A006490007EE0F4042566FE9000E7E08E00AA
:10643A00F5F0E884FF7E008F73EFC39410500CEFE1
:10644A008573F0A4FDACF08D7380037573FF900023
:10645A007EE0D39573400B90007EE0C39573F5718F
:10646A008003757100900102E0D395714006900196
:10647A0002E0F571900103E0C395715006900103A3
:10648A00E0F571807190007EE0C39566FE9000E7AA
:10649A00E08E00F5F0E884FF7E008F73EFC394105E
:1064AA00500CEF8573F0A4FDACF08D738003757307
:1064BA00FF85735B755A0090007EE0255BFFAE5A3C
:1064CA0050010E8E5A8F5B74FFBE0009D39F4005A0
:1064DA00855B7180037571FF900102E0D39571406D
:1064EA0006900102E0F571900103E0C39571500630
:1064FA00900103E0F571A20DB3B3500D90007FE057
:10650A00FE9000EFE0D39E5002800E740790005B6D
:10651A00F0E5B554BFF5B5802175A71075E700E51C
:10652A00CDC395714008E5B554BFF5B58006E5B50C
:10653A004440F5B575E71075A70075A700E56FC368
:10654A009409500AA2EDB34005C2ED123050AE5480
:10655A00AF557410C39F74279E400C90007DE0C312
:10656A00945A40030267DBA212B3400912421F7415
:10657A000690005BF0A223B34008E5B54404F5B5E4
:10658A008006E5B554FBF5B5A214B3500EE561D308
:10659A0094334007E561C394CC40028041900114D2
:1065AA00E0B40214120E26900085E075F050A4FFA4
:1065BA00AEF08E5C8F5D800F900090E075F050A475
:1065CA00FFAEF08E5C8F5DE55D455C6011E5B5441C
:1065DA0001F5B5742B90007CF012432FD214900071
:1065EA007DE0D394014007E561C3941A400280021A
:1065FA00C2149006D3E060031224EAA230300301E9
:10660A00B35017A230B34008E5B54408F5B5800683
:10661A00E5B554F7F5B5A23092039006D7E06003CA
:10662A001225C6A231300401B35017A231B3400873
:10663A00E5B54402F5B58006E5B554FDF5B5A231D8
:10664A0092049006DBE060031226B6A232300501FE
:10665A00B3500FA232B34004D2A28002C2A2A23225
:10666A0092059006DFE06003122792A233300601FA
:10667A00B3500FA233B34004D2A18002C2A1A23305
:10668A0092069006E3E0600312286EA234300701F6
:10669A00B35017A234B34008E5B54440F5B58006B7
:1066AA00E5B554BFF5B5A23492079006E7E060035A
:1066BA0012294AA235300801B35017A235B340084F
:1066CA00E5B54480F5B58006E5B5547FF5B5A23544
:1066DA0092089006EBE06003122A26A236300901DE
:1066EA00B3500FA236B34004D2878002C287A236C3
:1066FA0092099006EFE06003122B02A237300A01DA
:10670A00B3500FA237B34004D2908002C290A2378E
:10671A00920A9006F3E06003122BDEA238300B01D6
:10672A00B35017A238B34008E5B54410F5B5800652
:10673A00E5B554EFF5B5A238920B9006F7E0600381
:10674A00122CBAA239300C01B35017A239B340083F
:10675A00E5B54420F5B58006E5B554DFF5B5A239AF
:10676A00920C90007DE0C3945A5010E56FB4090969
:10677A0090007DE004F0756F00803BE56FB409037B
:10678A00756F00755500755400758D00758B007511
:10679A00640090007CE0C39441500890007CE004BF
:1067AA00F08006744190007CF090007CE0B44106D1
:1067BA00E5B554FEF5B590007DE0D394014007E5B8
:1067CA006AC3944140028009740E90005BF0124241
:0467DA001F024B50FF
:106874000000010001400160018001A001C001E0AD
:1068840002000300039603B603D603F404000500D4
:106894000512052405360548055A056C057E059044
:1068A40005A805C005DE0600061406280646066E81
:1068B40006AE05CF00FF013F015F017F019F01BFCD
:1068C40001DF01FF02FF039503B503D503F303FFC3
:1068D40004FF05110523053505470559056B057D9D
:1068E400058F05A705BF05CE05F106130627064546
:1068F400066D06AD06ED05DD0FAA0FA50F9F0F9AD5
:106904000F940F8D0F870F800F780F710F680F6032
:106914000F570F4E0F450F3B0F300F250F1A0F0E59
:106924000F020EF50EE80EDB0ECC0EBE0EAE0E9F61
:106934000E8E0E7D0E6C0E5A0E470E340E200E0C6B
:106944000DF70DE20DCB0DB50D9D0D850D6D0D549F
:106954000D3A0D200D050CE90CCE0CB10C940C76FF
:106964000C580C3A0C1B0BFB0BDB0BBB0B9A0B7977
:106974000B570B350B130AF10ACE0AAB0A870A64CC
:106984000A400A1C09F809D409B0098C09670943AB
:10699400091F08FB08D608B2088E086A08460823AF
:1069A40007FF07DC07B9079607730751072F070D81
:1069B40006EC06CA06AA068906690649062A060AD4
:1069C40005EC05CD05B0059205750558053C052077
:1069D400050504EA04CF04B5049C04820469045147
:1069E40004390422040B03F403DE03C803B2039D39
:1069F400038903750361034D033B03280316030452
:106A040002F202E102D102C002B002A002910282AB
:106A14000273026502570249023C022F0222021647
:106A2400020901FD01F201E601DB01D001C601BB4F
:106A340001B101A7019D0194018B018201790170CB
:106A440001680160015801500148014101390132D6
:106A5400012B0125011E01180111010B010500FF85
:106A640000FA0FA60FA00F990F920F8B0F840F7CC3
:106A74000F740F6B0F620F580F4E0F430F380F2C0C
:106A84000F1F0F120F050EF70EE80ED80EC80EB723
:106A94000EA50E930E800E6C0E580E420E2C0E1583
:106AA4000DFD0DE40DCB0DB10D950D790D5D0D3F73
:106AB4000D200D010CE10CC00C9E0C7C0C590C3506
:106AC4000C100BEA0BC40B9E0B760B4F0B260AFD26
:106AD4000AD40AAA0A800A550A2A09FF09D409A86D
:106AE400097C0950092508F908CD08A10875084A48
:106AF400081E07F307C8079D07730749072006F711
:106B040006CE06A6067E06570630060A05E405BF2D
:106B1400059B057705540532051004EF04CE04AE39
:106B2400048F047104530435041903FD03E203C7FD
:106B340003AD0394037B0363034B0334031E030875
:106B440002F302DE02CA02B602A30291027F026DC0
:106B5400025C024C023C022C021D020E020001F2F5
:106B640001E401D701CA01BE01B101A6019A018F56
:106B74000185017A01700166015D0153014A0141F9
:106B8400013901310129012101190112010B01040B
:106B940000FD00F700F000EA00E400DE00D900D3B5
:106BA40000CE00C900C400BF00BA00B500B100ADFA
:106BB40000A800A400A0009C009900950091008EFC
:0C6BC400008A008700840081007E007BB6
:10009E007547009007D0E4F0A3F07531007530007D
:1000AE00754D00754E00C23BD23C74FE9007D2F8DF
:1000BE00E4F0E8A3F074FE9007D4F8E4F0E8A3F0BF
:1000CE0074FE9007DEF0745A9007DFF0745A9007B2
:1000DE00E0F0D23DC22FC23FC23A22750B00750A24
:1000EE0000AE0AAF0BAC08AD09EDC39FEC9E4016F7
:1000FE0074FF126F7C75CF01780B740126F65004D5
:10010E0018E436F650DB22900057E0B4AA1C900794
:10011E008CE0B43C159007CCE0FEA3E0FFEF4E6000
:10012E0009741EBE0004D39F5003020243755D0086
:10013E00755C0075F8099007CCE0FEA3E0FF74072C
:10014E006F4E6006740E6F4E7006743A90078CF008
:10015E009007CCE0FEA3E0FF7408BE001ED39F40C4
:10016E001A7E017F089007CCE0FCA3E0FD1DBDFFC9
:10017E00011C1200038E5A8F5B801F9007CCE0FE8D
:10018E00A3E0FF7408126FE08F048E057E017F08D6
:10019E00CDCCCD1200038E5A8F5BAE5CAF5D740C6E
:1001AE00D39F74019E500302023EA2F9B3407EE536
:1001BE005D455C700375A382AE5CAF5D74016F4EDE
:1001CE00700375A300AE5CAF5D74026F4E700D9040
:1001DE0007CDE075F002A4FDACF08DA3AE5CAF5D73
:1001EE0074036F4E700375A300AE5CAF5D7403BEF7
:1001FE0000039F5013AC5AAD5BED2FFFEC3EFE900B
:10020E000088126FC3E0F5A3AE5CAF5DEFB40B09CF
:10021E00EEB401057414126F7CAE5CAF5DEFB40BDF
:10022E0007EEB4010375F80D785C126FF00201A8A9
:10023E00900057E4F022755D00755C0075F809902A
:10024E0007CCE0FEA3E0FF7408BE001ED39F401A49
:10025E007E017F089007CCE0FCA3E0FD1DBDFF01F1
:10026E001C1200038E5A8F5B801F9007CCE0FEA3FA
:10027E00E0FF7408126FE08F048E057E017F08CDBB
:10028E00CCCD1200038E5A8F5BAE5CAF5D7411D372
:10029E009F74019E5003020374A2F9B3500302032C
:1002AE0071E55D455C700375A3D2AE5CAF5D740104
:1002BE006F4E700375A300AE5CAF5D74026F4E702F
:1002CE000D9007CDE075F002A4FDACF08DA3AE5CF1
:1002DE00AF5D74036F4E700375A300AE5CAF5D74BB
:1002EE00046F4E700375A300AE5CAF5D74056F4E68
:1002FE00700375A300AE5CAF5D74066F4E70037530
:10030E00A300AE5CAF5D74076F4E700375A300AEB5
:10031E005CAF5D74086F4E700375A300AE5CAF5D8D
:10032E007408BE00039F5016AC5AAD5BED2FFFEC68
:10033E003EFE900083126FC3E5A3F075A300AE5C82
:10034E00AF5DEFB41009EEB401057414126F7CAEFC
:10035E005CAF5DEFB41007EEB4010375F80D785C79
:10036E00126FF002029722755D00755C0075F80938
:10037E00AE5CAF5D7417BE0004D39F500302044DF4
:10038E00A2F9B3500302044AE55D455C700375A300
:10039E00D2AE5CAF5D74016F4E700375A300AE5CA0
:1003AE00AF5D74026F4E700D9007CDE075F002A434
:1003BE00FDACF08DA3AE5CAF5D74036F4E70037534
:1003CE00A300AE5CAF5D74046F4E700375A300AEF8
:1003DE005CAF5D74056F4E700375A300AE5CAF5DD0
:1003EE0074066F4E700375A300AE5CAF5D74076F3D
:1003FE004E700375A300AE5CAF5D74086F4E700354
:10040E0075A300AE5CAF5D7408BE00039F500C90E8
:10041E000065126FC3E5A3F075A300AE5CAF5D740B
:10042E00166F4E70057414126F7CAE5CAF5D741651
:10043E006F4E700375F80D785C126FF002037E221A
:10044E00900057E0B4AB0280030204E8755D0075BE
:10045E005C0075F809AE5CAF5D7412BE007CD39F74
:10046E004078A2F9B34070E55D455C700375A382D8
:10047E00AE5CAF5D74016F4E700375A300AE5CAFE2
:10048E005D74026F4E700D9007CDE075F002A4FD05
:10049E00ACF08DA3AE5CAF5D74036F4E700375A3AD
:1004AE0000AE5CAF5D7403BE00039F500990006AFE
:1004BE00126FC3E0F5A3AE5CAF5D74116F4E7005A5
:1004CE007414126F7CAE5CAF5D74116F4E70037559
:1004DE00F80D785C126FF0020463229007DBE4F0F3
:1004EE0074649007CCF8E4F0E8A3F012037574C8B6
:1004FE009007CCF8E4F0E8A3F074FF900065F07478
:10050E00FF900066F074FF900067F0740090005F3B
:10051E00F074FF900068F0740090006AF07401901F
:10052E00006BF0900071E0B4371A90006EE090000E
:10053E0065F090006FE0900066F0900070E0900023
:10054E0067F080469007DB7401F074659007CCF875
:10055E00E4F0E8A3F012037574C89007CCF8E4F049
:10056E00E8A3F0900071E0B4371A90006EE09000AE
:10057E0065F090006FE0900066F0900070E09000E3
:10058E0067F0800674029007DBF09007DCE4F074ED
:10059E00669007CCF8E4F0E8A3F012037574C890E7
:1005AE0007CCF8E4F0E8A3F0900070E0B4371290B6
:1005BE00006EE090005FF090006FE0900068F080B9
:1005CE00769007DC7401F074679007CCF8E4F0E8DD
:1005DE00A3F012037574C89007CCF8E4F0E8A3F00A
:1005EE00900070E0B4371290006EE090005FF090D3
:1005FE00006FE0900068F0803E74029007DCF074AB
:10060E00689007CCF8E4F0E8A3F012037574C89074
:10061E0007CCF8E4F0E8A3F0900070E0B437129045
:10062E00006EE090005FF090006FE0900068F08048
:10063E000674039007DCF022E54E64046006E5992B
:10064E0064FF60028031A23B4004D23B8027E54E1E
:10065E00600874E6254E90005BF0E54D600874F07E
:10066E00254D90005BF0E54EB4010280FE754E0004
:10067E00754D00C23B8002C23BE54E90384AF828C9
:10068E002873754E00E599B4FF03754D01E599B4D5
:10069E00FE03754D02E599B4FD03754D03E599B45E
:1006AE00FC03754D04E599B4FA03754D05E599B44F
:1006BE00FB06754E0112421FE599B4F906754E04FC
:1006CE0012421FE599D394E54007E599C394F04093
:1006DE0002801685994F754E027E017F00E54FC34D
:1006EE0094E6126F9C8E328F339007D0E4F0A3F015
:1006FE00E599D394C44007E599C394E64002802857
:10070E0085994F754E0374E5C3954FF533753200D9
:10071E00AE32AF33906874126F6BE493F87401933A
:10072E009007D0C8F0A3C8F0D299020C5690006E74
:10073E00E07005A22DB3400280429007D0E0FEA3E8
:10074E00E0FF74FFBE00039F5009EFC39446EE9482
:10075E000640119007D0E0FEA3E0FFEFD3946DEEBC
:10076E00940640139007D0E0FEA3E0FF90008C1299
:10077E006FC3E599F0800385997480119007D0E0DE
:10078E00FEA3E0FF90008C126FC3E599F09007D0A6
:10079E00126FAA9007D0E0FEA3E0FFEFB40106EEC1
:1007AE00B4070280030209FD90078CE0B43C02807E
:1007BE00030209FDA22D50030208E8C29C90006EB0
:1007CE00E090012AF090006FE0900099F090007098
:1007DE00E09000B9F0900071E09000E2F0900072AD
:1007EE00E090008EF0900073E09000D4F0900074D2
:1007FE00E09000F2F0900075E09000C6F090007668
:10080E00E09000E4F0900077E0900114F090007812
:10081E00E0900178F0900079E0900179F090007A04
:10082E00E090017AF0123BE0900080E09000FBF047
:10083E00900081E09000B2F0900082E09000B3F062
:10084E0074639007CCF8E4F0E8A3F074AB90005713
:10085E00F012044E900057E4F07464F50975080028
:10086E001200E9A2224039757301E573D394075043
:10087E002DE5739007CCF8E4F0E8A3F074AA90008D
:10088E0057F0120115E573C39407500A7464F50905
:10089E007508001200E97873740126F650CC803783
:1008AE00757308E573D3940E502DE5739007CCF84D
:1008BE00E4F0E8A3F074AA900057F0120115E57366
:1008CE00C3940E500A7464F5097508001200E97895
:1008DE0073740126F650CC0209E7C29C90012AE0FF
:1008EE0090006EF0900099E090006FF09000B9E0EB
:1008FE00900070F09000E2E0900071F090008EE0B9
:10090E00900072F09000D4E0900073F09000F2E04E
:10091E00900074F09000C6E0900075F09000E4E056
:10092E00900076F0900114E0900077F07400900043
:10093E0078F07400900079F0740090007AF074638F
:10094E009007CCF8E4F0E8A3F074AB900057F012E7
:10095E00044E900057E4F07464F509750800120017
:10096E00E9757301E573D394075026E5739007CCB0
:10097E00F8E4F0E8A3F074AA900057F01201157491
:10098E0064F5097508001200E97873740126F650B3
:10099E00D3D29C7599FB743C90078CF0757308E567
:1009AE0073D3940E5026E5739007CCF8E4F0E8A3C9
:1009BE00F074AA900057F01201157464F5097508C9
:1009CE00001200E97873740126F650D374C89007AC
:1009DE00CCF8E4F0E8A3F080FE74C89007CCF8E4FD
:1009EE00F0E8A3F0D29C754E00754D007599FB0290
:1009FE000C569007D0E0FEA3E0FFEF4E70068599EF
:100A0E00317530009007D0E0FEA3E0FF74016F4E09
:100A1E00701BAC30AD31AA32AB33ED2BFBEC3AFA96
:100A2E008A068B0790008C126FC3E599F09007D061
:100A3E00126FAA9007D0E0FEA3E0FF74026F4E7013
:100A4E0021AC30AD3174566D4C7006E54F64E660E6
:100A5E0002800312421F123BE0854F99754E0075BE
:100A6E004D00020C569007D0E0FEA3E0FF90008CE4
:100A7E00126FC3E599F09007D0126FAA9007D0E0DD
:100A8E00FEA3E0FFAC32AD338F028E038C068D07D2
:100A9E009068B8126F6BE493F9740193FEEAD39EDB
:100AAE00EB994009854F99754E00754D00020C5615
:100ABE009007D0E0FEA3E0FF90008C126FC3E59983
:100ACE00F09007D0126FAA9007D0E0FEA3E0FFEFE0
:100ADE00B40006EEB401028003020C56900067E0EB
:100AEE00D394C7400B900067E0C394C8F550801AAA
:100AFE00900067E0D39463400B900067E0C394646A
:100B0E00F5508006900067E0F550E55075F002A4B0
:100B1E00FFAEF08F73EF90008C126FCEEFFCE0FD06
:100B2E00EC90008F126FCEEDFCE0FDEC2DB5500277
:100B3E008003020C470FEF90008C126FCEE573FF0F
:100B4E00E0FCEF900090126FCEECFFE0FCEFC39C48
:100B5E00B550028003020C47E57390008E126FCEE3
:100B6E00E573FFE0FCEF900091126FCEECFFE0FC1E
:100B7E00EF2CB550028003020C47E57390009212E1
:100B8E006FCEE0C3955090006EF0E5739000931217
:100B9E006FCEE0C3955090006FF0E5739000941205
:100BAE006FCEE0C39550900070F07400900071F01D
:100BBE0074FF900072F0E573900096126FCEE0C352
:100BCE009550900073F0E573900097126FCEE0C3CE
:100BDE009550900074F0E573900098126FCEE0C3BC
:100BEE009550900075F0E573900095126FCEE0C3AE
:100BFE0095509007CCF8E4F0E8A3F074AB90005752
:100C0E00F012044E7464F5097508001200E990079D
:100C1E00CC126FAA12044E7464F509750800120006
:100C2E00E99007CC126FAA12044E7599F97464F507
:100C3E00097508001200E980FE7599FF7464F509C4
:080C4E007508001200E980FEA8
:0F384A0002069002073B020A00020A73020ABE3E
:100C560022E54D903859F8282873020D699007D07F
:100C6600E0FEA3E0FF90005D126FC3E0F5999007E8
:100C7600D0126FAA9007D0E0FEA3E0FF74116F4E6A
:100C86007003754D00020D69856E99020D69900716
:100C9600D0E0FEA3E0FF90008C126FC3E0F599EF61
:100CA600B40107EEB40703754D009007D0126FAA82
:070CB600020D699007D1E077
:0F385900020C60020C63020C8E020C94020CB97C
:100CBD00903A0CF8282873855399020D5E855F993B
:100CCD00020D5E856199020D5E856599020D5E8549
:100CDD006799807D85689980788569998073856A23
:100CED0099806E90001EE0F5998066A23CB3400796
:100CFD007599FAC23C8041A22CB3400575990F80BD
:100D0D00359007DBE0600A9007DBE024DCF5998085
:100D1D00169007DCE0600A9007DCE024DEF5998090
:100D2D000690005BE0F59990005BE4F09007DBE442
:100D3D00F09007DCE4F0C22C8017856B998012854A
:100D4D006699800D856C9980087599FC8003754DA9
:010D5D000095
:103A0C00020CC4020CCA020CD0020CD6020CDC0252
:103A1C000CE1020CE6020CEB020CF0020CF8020DAD
:0D3A2C0047020D4C020D51020D56020D5BBC
:0B0D5E009007D0126FAA8003123A39F0
:03386800020D66E8
:100D690022E537255BFFAE5A50010E90008C126FB9
:100D7900C3E0F538E537255BFFAE5A50010E0FBFCA
:100D890000010E90008C126FC3E0F539853F3BE5F9
:100D990038B539058538378041E539D39538401D4F
:100DA900E539C39538853AF0A4FFAEF0E53B8E04EA
:100DB9008F05FF126F8CED2538F537801DE538C397
:100DC9009539853AF0A4FFAEF0E53B8E048F05FF17
:100DD900126F8CEDF4042538F53722E539D39538AF
:100DE900401DE539C39538853AF0A4FFAEF0E53BDF
:100DF9008E048F05FF126F8CED2538F537801DE5C0
:100E090038C39539853AF0A4FFAEF0E53B8E048FDF
:100E190005FF126F8CEDF4042538F5372290009206
:100E2900E0B40170E56775F00A84FF7E008F37E54D
:100E39006775F00A84ADF07C008D3A753F0A755AE2
:100E490005755B24E537C394115005120D6A8006B8
:100E59009005C1E0F537E537900085F0E56775F055
:100E69000A84FF7E008F37E56775F00A84ADF07C50
:100E7900008D3A753F0A755A05755B5AE537C39473
:100E8900115005120D6A80069005F7E0F537E53730
:100E9900900016F022900092E0B4016AE56775F0BF
:100EA9000A84FF7E008F37E56775F00A84ADF07C10
:100EB900008D3A753F0A755A05755B36E537C39457
:100EC900115005120D6A80069005D3E0F537853774
:100ED9004BE56775F00A84FF7E008F37E56775F08B
:100EE9000A84ADF07C008D3A753F0A755A05755B29
:100EF90048E537C394115005120D6A80069005E53F
:100F0900E0F53785374C22E55F75F00484FF7E00F4
:100F19008F37E55F75F00484ADF07C008D3A753F3D
:100F290004755A01755B00E537C3943F5005120DEE
:100F39006A80069001CBE0F537853729752800903E
:100F4900005AE075F020A4FFAEF09000DDE08E04B9
:100F59008F05FF126F8C8D379000C5E0D3955F50D8
:100F6900030210169000E9E0D3955F4010ED90015F
:100F7900CC126FCEE0F52B752A000210139000B445
:100F8900E0D3955F4043E5379001CC126FCEE0F591
:100F990038E5379001EC126FCEE0F5399000E9E0C1
:100FA900F404255FF53A9000B4E0FE9000E9E0F41E
:100FB900042EF53BE538B539058538378003120D20
:100FC900E485372B752A008041E5379001EC126FD3
:100FD900CEE0F538E53790020C126FCEE0F5399086
:100FE90000B4E0F404255FF53A9000C5E0FE9000F6
:100FF900B4E0F4042EF53BE538B53905853837807A
:1010090003120DE485372B752A000210BD9000EC00
:10101900E0D3955F5011E53790024C126FCEE0F5A1
:101029002B752A000210BD9000B5E0D3955F50439F
:10103900E53790022C126FCEE0F538E53790024C77
:10104900126FCEE0F5399000B5E0F404255FF53A6A
:101059009000ECE0FE9000B5E0F4042EF53BE53895
:10106900B539058538378003120DE485372B752A84
:10107900008041E53790020C126FCEE0F538E53774
:1010890090022C126FCEE0F5399000C5E0F40425EA
:101099005FF53A9000B5E0FE9000C5E0F4042EF546
:1010A9003BE538B539058538378003120DE48537B6
:1010B9002B752A00229000FDE0F53C753F11755A09
:1010C90002755B00AE52AF53E53C75F00FA4FDAC61
:1010D900F0EDD39FEC9E4021E53C8E048F05FF1275
:1010E9006F8CED75F010A4FFAEF0E55F75F011841B
:1010F900FD7C00ED2FF53D800EE55F75F01184FF55
:101109007E00EF24F0F53D853D37E55F75F01184EC
:10111900AFF07E008F3A120D6A85373EAE52AF535B
:101129009000FDE075F00FA4FDACF0EDD39FEC9EAF
:101139004028755A02755B10853D37120D6A853E48
:1011490038853739AE52AF53E53C8E048F05FF120F
:101159006FB78D3A853C3B120DE485372975280018
:10116900752B64752A00229000FDE0F53C753F114E
:10117900755A02755B00AE52AF53E53C75F00FA48A
:10118900FDACF0EDD39FEC9E4021E53C8E048F052C
:10119900FF126F8CED75F010A4FFAEF0E56175F0EC
:1011A9001184FD7C00ED2FF53D800EE56175F01190
:1011B90084FF7E00EF24F0F53D853D37E56175F04C
:1011C9001184AFF07E008F3A120D6A85373EAE5218
:1011D900AF539000FDE075F00FA4FDACF0EDD39F87
:1011E900EC9E4028755A02755B10853D37120D6AD1
:1011F900853E38853739AE52AF53E53C8E048F05AD
:10120900FF126FB78D3A853C3B120DE4853729757E
:101219002800E56B6017E56BC394FE50109000F150
:10122900E0B402099000DFE0D3940B50028017AEBE
:1012390028AF29E56B126F9C74E78E048F05FF12A6
:101249006F8C8C288D299000C7E0B40453E55F7535
:10125900F00484FF7E008F37E55F75F00484ADF0FC
:101269007C008D3A753F04755A01755B00E537C3FB
:10127900943F5005120D6A80069001CBE0F537AE18
:1012890028AF29E537126F9C74648E048F05FF120D
:101299006F8CAE28AF29EF2DFDEE3CFC8C288D29F3
:1012A900752B64752A0022900092E0B40146E56727
:1012B90075F00A84FF7E008F37E56775F00A84AD03
:1012C900F07C008D3A753F0A755A05755B00E53764
:1012D900C394115005120D6A800690059DE0F537FB
:1012E900AE2AAF2BE5372FFF50010E7464126FE061
:1012F9008E2A8F2B900093E0B40146E56875F00AB9
:1013090084FF7E008F37E56875F00A84ADF07C00B4
:101319008D3A753F0A755A05755B6CE537C39411AB
:101329005005120D6A8006900609E0F537AE2AAF1E
:101339002BE5372FFF50010E7464126FE08E2A8F50
:101349002B9000A2E0B40249E56AC3944175F00507
:1013590084FF7E008F37E56A75F00584ADF07C0067
:101369008D3A753F05755A06755B00E537C39413C9
:101379005005120D6A800690069FE0F537AE2AAF38
:101389002BE5372FFF50010E7464126FE08E2A8F00
:101399002B9000E4E0B40202800302144FE55F756C
:1013A900F01584FF7E008F37E55F75F01584ADF089
:1013B9007C008D3A753F15755A03755BF4E537C3A3
:1013C900940B5005120D6A800690048BE0F537E501
:1013D9003775F0FFA4FFAEF09000E5E08E048F05AD
:1013E900FF126F8CED90007EF0E56675F078A4FF32
:1013F900AEF074FF8E048F05FF126F8C8C5A8D5BD3
:1014090074028C068D071200398F37AC5AAD5B74A4
:1014190004FF126FB78D3A753F04755A06755B283C
:10142900E537C3941D5005120D6A80069006D1E078
:10143900F537AE2AAF2BE5372FFF50010E74641232
:101449006FE08E2A8F2B900091E0B4025DE5617503
:10145900F064A4FFAEF074081200398E5C8F5D74DD
:10146900058E048F05FF126F8C8D37AE5CAF5D74EE
:10147900058E048F05FF126FB78D3A753F05755AB2
:1014890005755BDEE537C394135005120D6A8006B6
:1014990090067DE0F537AE2AAF2BE5372FFF5001D7
:1014A9000E7464126FE08E2A8F2B9000D3E0703C8B
:1014B90090005AE075F00584FF7E008F3790005A3E
:1014C900E075F00584ADF07C008D3A753F05755ADD
:1014D90005755BC0E537C3941D5005120D6A80067A
:1014E900900669E0F537E537900086F02290009A7A
:1014F900E0B401179007D7E0252BFFAE2A50010E63
:101509009000EEE0126FE08E2A8F2B900112E0B46A
:101519000114900113E0A852B8000495535007E54F
:101529005FC39560400280129000BCE0252BFFAE9E
:101539002A50010E8E2A8F2B802F90009AE0B40337
:1015490016A22FB3B350109007DAE0C39405A8523E
:10155900B800069553400280109000BCE0252BFF8F
:10156900AE2A50010E8E2A8F2B900094E0B402020D
:1015790080030218F4900097E0602FE567D3944642
:101589004028900017E0FEA3E0FF9000D2E075F03C
:1015990003A4FDACF0EFD39DEE9C400E9000F6E065
:1015A900A852B80005D3955350030218F49000C708
:1015B900E0B40302800302175885615B755A0090F5
:1015C900009EE0A852B800049553500E90009FE089
:1015D900A85AB80005D3955B5003021755E5617504
:1015E900F002A4FFAEF074158E048F05FF126F8C04
:1015F9008C068D0790061C126FC3FEE0FFEE90006B
:1016090096E0FEEF8E0088F0A4FFAEF074648E04BD
:101619008F05FF126F8C8C5A8D5B90005AE075F024
:1016290018A4FFAEF09000DDE08E048F05FF126F65
:101639008C8C068D07900634126FC3AE5AAF5BE0EF
:10164900126F9C74648E048F05FF126F8C8C5A8DF7
:101659005BE565A85AB80077D3955B4072E565C329
:10166900955BFFE4955AFE8E5A8F5B7428BE000382
:101679009F500C755B28755A00740D90005BF0AE95
:101689005AAF5B900097E0126F9C74288E048F0507
:10169900FF126F8C8C5A8D5BAE28AF29740A8E04A9
:1016A9008F05FF126F8C8D068C07AC5AAD5BCFCEC0
:1016B900CF120003740A8E048F05FF126F8C8C5AA7
:1016C9008D5BAE28AF29126FE88E288F29807DE5C2
:1016D90065A85AB80004955B5072AE5AAF5BE565D0
:1016E900126FE08E5A8F5B7428BE00039F500C75F1
:1016F9005B28755A00740D90005BF0AE5AAF5B9091
:101709000097E0126F9C74288E048F05FF126F8C6E
:101719008C5A8D5BAE28AF29740A8E048F05FF128F
:101729006F8C8D068C07AC5AAD5BCFCECF12000300
:10173900740A8E048F05FF126F8C8C5A8D5BAE284C
:10174900AF29EF2DFDEE3CFC8C288D290218F49071
:1017590000DFE0855FF0A4FFAEF07405126F9C74A2
:10176900071200398E5A8F5B90009EE0A852B8008C
:10177900049553501290009FE075F002A4FDACF05F
:10178900EFC39DEE9C40030218F4E55F75F00B84EE
:10179900FF7E0090061C126FC3FEE0FFEE900096DC
:1017A900E0FEEF8E0088F0A4FFAEF074648E048F23
:1017B90005FF126F8C8C5A8D5B90005AE075F018FA
:1017C900A4FFAEF09000DDE08E048F05FF126F8C50
:1017D9008C068D07900634126FC3AE5AAF5BE012C8
:1017E9006F9C74648E048F05FF126F8C8C5A8D5B0D
:1017F900E565A85AB80077D3955B4072E565C3954E
:101809005BFFE4955AFE8E5A8F5B7428BE00039FD6
:10181900500C755B28755A00740D90005BF0AE5A38
:10182900AF5B900097E0126F9C74288E048F05FFC0
:10183900126F8C8C5A8D5BAE28AF29740A8E048F77
:1018490005FF126F8C8D068C07AC5AAD5BCFCECFDE
:10185900120003740A8E048F05FF126F8C8C5A8D47
:101869005BAE28AF29126FE88E288F29807DE56548
:10187900A85AB80004955B5072AE5AAF5BE5651281
:101889006FE08E5A8F5B7428BE00039F500C755B06
:1018990028755A00740D90005BF0AE5AAF5B90004A
:1018A90097E0126F9C74288E048F05FF126F8C8C41
:1018B9005A8D5BAE28AF29740A8E048F05FF126F0B
:1018C9008C8D068C07AC5AAD5BCFCECF120003745A
:1018D9000A8E048F05FF126F8C8C5A8D5BAE28AF70
:1018E90029EF2DFDEE3CFC8C288D29229000F2E099
:1018F900B4026AE55F75F00884FF7E008F37E55F03
:1019090075F00884ADF07C008D3A753F08755A0171
:10191900755BE0E537C3943F5005120D6A80069068
:10192900028BE0F53785372D752C00AE2CAF2DAC29
:101939002AAD2B12000374648E048F05FF126F8C7D
:101949008C2C8D2D90008FE08C068D07126F9C7466
:10195900648E048F05FF126F8C8C2C8D2DAE28AFF1
:1019690029AC2AAD2B12000374648E048F05FF1273
:101979006F8C8C288D2990008FE08C068D07126F53
:101989009C74648E048F05FF126F8C8C288D29A29C
:101999000D401DAE52AF537405BE00039F5002D2D5
:1019A9000DE561D394CC4008D201741190005BF02D
:1019B9009000F1E0B402089000DFE0640B6002805F
:1019C90035AE28AF29E56B126F9C74E78E048F053D
:1019D900FF126F8C8C288D299000F2E0B40217AEAB
:1019E9002CAF2DE56B126F9C74E78E048F05FF12E7
:1019F9006F8C8C2C8D2D9000B1E05402601B9000EF
:101A0900A8E0A852B80012D39553400DA20DB3B364
:101A19005007E561C3949A40028028AE34AF3590EF
:101A290000A6E075F002A4FDACF0EF2DFDEE3CFC44
:101A390074022DFD50010CE561BC0007D39D4003E4
:101A4900754301856135753400E5437003021B3820
:101A5900900104E0C395435003021B2A900114E04E
:101A6900C394025076E56775F00A84FF7E009005FD
:101A79008C126FC3E0F55B755A00AE5AAF5B9000EC
:101A8900A7E0126F9C74648E048F05FF126F8C8C13
:101A99005C8D5D900104E004C395438C068D0712AB
:101AA9006F9C900104E08E048F05FF126F8C8C5C93
:101AB9008D5DAE28AF29EF2DFDEE3CFC8C288D29DC
:101AC9009000F2E0B40212AE2CAF2DAA5CAB5DEF30
:101AD9002BFBEE3AFA8A2C8B2D8046900104E00408
:101AE900C39543854BF0A4FFAEF0900104E08E044A
:101AF9008F05FF126F8C8C5C8D5DAE28AF29EF2DA1
:101B0900FDEE3CFC8C288D299000F2E0B40212AE67
:101B19002CAF2DAA5CAB5DEF2BFBEE3AFA8A2C8B2E
:101B29002D0543900104E0C395435003754300908C
:101B390000B1E05401601B9000A5E0A852B8001262
:101B4900D39553400DA20DB3B35007E55FC394CCB1
:101B5900400280259000A3E075F003A4FFAEF0E5F4
:101B6900402FFF50010E74032FFF50010EE55FBE99
:101B79000007D39F4003754401855F40E544700326
:101B8900021C6B900105E0C395445003021C5D9053
:101B99000114E0C394025076E56775F00A84FF7E6C
:101BA9000090058C126FC3E0F55B755A00AE5AAF11
:101BB9005B9000A4E0126F9C74648E048F05FF1281
:101BC9006F8C8C5C8D5D900105E004C395448C0697
:101BD9008D07126F9C900105E08E048F05FF126F2F
:101BE9008C8C5C8D5DAE28AF29EF2DFDEE3CFC8C15
:101BF900288D299000F2E0B40212AE2CAF2DAA5C18
:101C0900AB5DEF2BFBEE3AFA8A2C8B2D80469001C7
:101C190005E004C39544854CF0A4FFAEF09001059E
:101C2900E08E048F05FF126F8C8C5C8D5DAE28AF42
:101C390029EF2DFDEE3CFC8C288D299000F2E0B4B3
:101C49000212AE2CAF2DAA5CAB5DEF2BFBEE3AFA7C
:101C59008A2C8B2D0544900105E0C39544500375EA
:101C69004400900107E02529FFAE2850010E8E2877
:101C79008F299000B6E0A828B8000495295009904A
:101C890000B6E0F5297528009000F2E0B4020D9045
:101C990000B6E0A82CB80006952D400280099000F6
:101CA900B6E0F52D752C00229000F2E0B401028017
:101CB90003021DBCA20DB35003021DBA9000BDE082
:101CC900B40168AE28AF29AC52AD53120003743C7D
:101CD9008E048F05FF126F8C9000CDE0BC00109D23
:101CE900400D9000CFE0A828B8000495295002D2F1
:101CF90002AE28AF29AC52AD53120003743C8E04D6
:101D09008F05FF126F8C9000CDE0C3940ABC0015BB
:101D1900D39D40119000CFE0C39405A828B80005D1
:101D2900D3952950028002C2028068AE28AF29AC3F
:101D390052AD5312000374788E048F05FF126F8C15
:101D49009000CDE0BC00109D400D9000CFE0A82888
:101D5900B8000495295004D2028038AE28AF29ACC6
:101D690052AD5312000374788E048F05FF126F8CE5
:101D79009000CDE0C3940ABC0015D39D401190009A
:101D8900CFE0C39405A828B80005D395295002804F
:101D990002C202A202B34019AE28AF299000CEE0D8
:101DA900126F9C74648E048F05FF126F8C8C288DC2
:101DB900298002C202A200B34006A201B3B35009AE
:101DC90090001DE4F0A3F08024AE28AF297400D35D
:101DD9009F74019E400C90001DE528F0A3E529F0B1
:101DE900800B74FF90001DF8E4F0E8A3F09000D494
:101DF900E0D39402400C9000BFE07006A20DB3B38B
:101E09004002801AAE28AF297402126F9C8E288F67
:101E190029AE2CAF2D7402126F9C8E2C8F2D900041
:101E2900BDE0B4011AAE28AF297402126F9C8E2846
:101E39008F29AE2CAF2D7402126F9C8E2C8F2DAE74
:101E490028AF29745E126F9C740A8E048F05FF12E5
:101E59006F8C8C288D299000F2E0B40217AE2CAF5C
:101E69002D745E126F9C740A8E048F05FF126F8C9D
:101E79008C2C8D2DAE28AF297402BE000AD39F4049
:101E890006752902752800AE2CAF2D7402BE000A12
:101E9900D39F4006752D02752C0090001BE528F094
:101EA900A3E529F02290005AE090038C126FCEE04E
:101EB900F54175426490005AE0FE9000C8E0D39E57
:101EC9004037E55F75F00884FF7E008F37E55F7561
:101ED900F00884ADF07C008D3A753F08755A03759A
:101EE9005B96E537C3941F5005120D6A800690046E
:101EF90041E0F5378537428035E55F75F00884FFA5
:101F09007E008F37E55F75F00884ADF07C008D3A6F
:101F1900753F08755A03755BB6E537C3941F5005BD
:101F2900120D6A8006900461E0F5378537422290E8
:101F390000FEE0F53C753F11755A04755B00AE5221
:101F4900AF53E53C75F00FA4FDACF0EDD39FEC9ECB
:101F59004021E53C8E048F05FF126F8CED75F01062
:101F6900A4FFAEF0E55F75F01184FD7C00ED2FF55F
:101F79003D800EE55F75F01184FF7E00EF24F0F5DA
:101F89003D853D37E55F75F01184AFF07E008F3AEE
:101F9900120D6A85373EAE52AF539000FEE075F0E0
:101FA9000FA4FDACF0EDD39FEC9E4028755A047543
:101FB9005B10853D37120D6A853E38853739AE523B
:101FC900AF53E53C8E048F05FF126FB78D3A853C00
:101FD9003B120DE4853741754264229000FEE0F51D
:101FE9003C753F11755A04755B00AE52AF53E53C21
:101FF90075F00FA4FDACF0EDD39FEC9E4021E53CBC
:102009008E048F05FF126F8CED75F010A4FFAEF0F2
:10201900E56175F01184FD7C00ED2FF53D800EE53D
:102029006175F01184FF7E00EF24F0F53D853D37A1
:10203900E56175F01184AFF07E008F3A120D6A8563
:10204900373EAE52AF539000FEE075F00FA4FDACE1
:10205900F0EDD39FEC9E4028755A04755B10853DC1
:1020690037120D6A853E38853739AE52AF53E53C94
:102079008E048F05FF126FB78D3A853C3B120DE434
:102089008537417542649000C7E0B4047990005ADD
:10209900E0FE9000C8E0D39E4037E55F75F0088404
:1020A900FF7E008F37E55F75F00884ADF07C008D09
:1020B9003A753F08755A03755B96E537C3941F5007
:1020C90005120D6A8006900441E0F5378537428094
:1020D90035E55F75F00884FF7E008F37E55F75F0A1
:1020E9000884ADF07C008D3A753F08755A03755B1D
:1020F900B6E537C3941F5005120D6A800690046136
:10210900E0F53785374222900092E0B4013BE5675C
:1021190075F00A84FF7E008F37E56775F00A84AD94
:10212900F07C008D3A753F0A755A05755B12E537E3
:10213900C394115005120D6A80069005AFE0F5377A
:10214900E5422537C39464F542900093E0B4013B1E
:10215900E56875F00A84FF7E008F37E56875F00A37
:1021690084ADF07C008D3A753F0A755A05755B7E22
:10217900E537C394115005120D6A800690061BE0DD
:10218900F537E5422537C39464F542E5412542F523
:102199003690009AE0B402109007D6E02536FE90FA
:1021A90000EEE0F4042EF5369000F1E0D3940140FE
:1021B90040E56BC394E7501D74E7C3956BFE900728
:1021C900D8E08E00F5F0E884FF7E008F37E53625EC
:1021D90037F536801CE56BC394E7FE9007D8E08E8F
:1021E90000F5F0E884FF7E008F37E536C39537F5B3
:1021F90036A20D4006E5412464F536E536D39464EC
:102209004009E536C39464F53680037536009000BD
:10221900CAE0C3953650069000CAE0F53622D200CE
:10222900900084E0A852B80004955350419000846E
:10223900E0A852B800049553500375360F900084F6
:10224900E004A852B800049553500375360A90006B
:1022590084E02402A852B800049553500575360548
:10226900C200900084E06006740990005BF0C23FF0
:102279007E017F009000D0E0126F9C9000DFE08E1D
:10228900048F05FF126F8CE55FBC0017D39D4013C7
:102299009000D9E0B40204D23F8002C200740A90CF
:1022A900005BF09000D1E0C3956750159000E3E022
:1022B900A852B8000495535002C200740B90005BF9
:1022C900F0E567C39464501D900129E0600D900109
:1022D90029E0A852B80006955340028008C200744C
:1022E9000B90005BF0A2004003753605900112E0E7
:1022F900B40114900113E0A852B800049553500793
:10230900E55FC39560400280089000BBE0F5368028
:102319003A90009AE0B40306A22FB3B34002802B8F
:102329009007DAE0C39405A852B800049553500CFD
:102339009000BBE0F536740C90005BF09007DAE092
:10234900A852B8000495535002C20085366C90001B
:102359008CE02536FE90005AE075F01E84FC7F0063
:10236900EE2CF5362290005AE075F00584FF7E00C8
:102379008F3790005AE075F00584ADF07C008D3AF6
:10238900753F05755A03755BD69000DDE01475F04D
:102399000584FF7E00E537BE00039F5005120D6AD4
:1023A900800BE537900462126FCEE0F537E5379080
:1023B90007D9F09007D9E0FE9000CCE0C39E500801
:1023C9009000CCE09007D9F022E56775F00A84FF08
:1023D9007E0090058C126FC3E0F546E546D3946400
:1023E9004010E546C3946475F00F84FF7E008F4664
:1023F90080037546009000AFE02546F5462290001F
:10240900C7E0C3940350269007C6E0FEA3E0FF741B
:1024190004120039E55F126F9C740F8E048F05FF5B
:10242900126F8C9007C4ECF0A3EDF080249007C6DE
:10243900E0FEA3E0FF7404120039E561126F9C7499
:102449000F8E048F05FF126F8C9007C4ECF0A3ED7B
:10245900F09000A2E0B40262E56AC3944175F00508
:1024690084FF7E008F37E56A75F00584ADF07C0046
:102479008D3A753F05755A06755B14E537C3941790
:102489005005120D6A80069006B3E0F5379007C42F
:10249900E0FEA3E0FF740A8E048F05FF126F8CE53E
:1024A900378C068D07126F9C740A8E048F05FF12F4
:1024B9006F8C9007C4ECF0A3EDF09007C4E0FEA385
:1024C900E0FF9007CAE0FCA3E0FDEDD39FEC9E403E
:1024D9000F9007CAE0F8A3E09007C4C8F0A3C8F0BA
:1024E900229006D3E090386BF8282873804C8553E6
:1024F9007380479000DFE0855FF0A4FFAEF07408B9
:102509001200398F738033856173802E85677380DC
:10251900298568738024856973801F856A73801A89
:10252900856B7380158566738010856573800B854F
:0A2539006C73800690001EE0F5733D
:10386B000224F50224F70224FC022510022515027E
:10387B00251A02251F02252402252902252E0225A1
:07388B003302253802253D40
:102543009006D4E0FE9006D5E0D39E404B9006D390
:10255300E0B404189006D5E0C395735002D23090CE
:1025630006D4E0D395734002C230802A9006D4E0AB
:10257300C3957350099006D5E0D39573500280023A
:10258300D2309006D4E0D3957350099006D5E0C3BA
:1025930095735002C230802A9006D4E0D3957340DD
:1025A300099006D5E0C3957340028002C2309006BD
:1025B300D4E0C3957340099006D5E0D395734002E8
:1025C300D230229006D7E0903892F8282873804CB6
:1025D30085537380479000DFE0855FF0A4FFAEF082
:1025E30074081200398F738033856173802E856779
:1025F3007380298568738024856973801F856A7356
:10260300801A856B7380158566738010856573806A
:0C2613000B856C73800690001EE0F573D0
:103892000225D10225D30225D80225EC0225F10208
:1038A20025F60225FB02260002260502260A02262A
:0738B2000F02261402261983
:10261F009006D8E0FE9006D9E0D39E405F9006D793
:10262F00E0B404189006D9E0C395735002D23190EC
:10263F0006D8E0D395734002C231803E9006D8E0B1
:10264F00C3957350099006D9E0D395735002800259
:10265F00D2319006D8E0D3957350099006D9E0C3D4
:10266F0095735002C2319006D7E0B401099000EB88
:10267F00E0D3956150028002C231802A9006D8E0E3
:10268F00D3957340099006D9E0C395734002800239
:10269F00C2319006D8E0C3957340099006D9E0D3B4
:1026AF0095734002D231229006DBE09038B9F828BA
:1026BF002873804C85537380479000DFE0855FF06F
:1026CF00A4FFAEF074081200398F738033856173E5
:1026DF00802E856773802985687380248569738050
:1026EF001F856A73801A856B7380158566738010DA
:1026FF00856573800B856C73800690001EE0F57303
:1038B9000226C10226C30226C80226DC0226E1022C
:1038C90026E60226EB0226F00226F50226FA022651
:0738D900FF0227040227098A
:10270F009006DCE0FE9006DDE0D39E404B9006DBAA
:10271F00E0B404189006DDE0C395735002D23290F6
:10272F0006DCE0D395734002C232802A9006DCE0CB
:10273F00C3957350099006DDE0D395735002800264
:10274F00D2329006DCE0D3957350099006DDE0C3DA
:10275F0095735002C232802A9006DCE0D395734005
:10276F00099006DDE0C3957340028002C2329006E5
:10277F00DCE0C3957340099006DDE0D3957340020A
:10278F00D232229006DFE09038E0F8282873804C90
:10279F0085537380479000DFE0855FF0A4FFAEF0B4
:1027AF0074081200398F738033856173802E8567AB
:1027BF007380298568738024856973801F856A7388
:1027CF00801A856B7380158566738010856573809D
:0C27DF000B856C73800690001EE0F57303
:1038E00002279D02279F0227A40227B80227BD02B4
:1038F00027C20227C70227CC0227D10227D60227D8
:07390000DB0227E00227E5CE
:1027EB009006E0E0FE9006E1E0D39E404B9006DFC2
:1027FB00E0B404189006E1E0C395735002D2339015
:10280B0006E0E0D395734002C233802A9006E0E0E5
:10281B00C3957350099006E1E0D395735002800283
:10282B00D2339006E0E0D3957350099006E1E0C3F4
:10283B0095735002C233802A9006E0E0D395734023
:10284B00099006E1E0C3957340028002C233900603
:10285B00E0E0C3957340099006E1E0D39573400225
:10286B00D233229006E3E0903907F8282873804C86
:10287B0085537380479000DFE0855FF0A4FFAEF0D7
:10288B0074081200398F738033856173802E8567CE
:10289B007380298568738024856973801F856A73AB
:1028AB00801A856B738015856673801085657380C0
:0C28BB000B856C73800690001EE0F57326
:1039070002287902287B022880022894022899023B
:10391700289E0228A30228A80228AD0228B202285E
:07392700B70228BC0228C111
:1028C7009006E4E0FE9006E5E0D39E404B9006E3D9
:1028D700E0B404189006E5E0C395735002D2349033
:1028E70006E4E0D395734002C234802A9006E4E000
:1028F700C3957350099006E5E0D3957350028002A3
:10290700D2349006E4E0D3957350099006E5E0C30E
:1029170095735002C234802A9006E4E0D395734041
:10292700099006E5E0C3957340028002C234900621
:10293700E4E0C3957340099006E5E0D39573400240
:10294700D234229006E7E090392EF8282873804C7D
:1029570085537380479000DFE0855FF0A4FFAEF0FA
:1029670074081200398F738033856173802E8567F1
:102977007380298568738024856973801F856A73CE
:10298700801A856B738015856673801085657380E3
:0C2997000B856C73800690001EE0F57349
:10392E0002295502295702295C02297002297502C3
:10393E00297A02297F02298402298902298E0229E5
:07394E009302299802299D54
:1029A3009006E8E0FE9006E9E0D39E404B9006E7F0
:1029B300E0B404189006E9E0C395735002D2359051
:1029C30006E8E0D395734002C235802A9006E8E01A
:1029D300C3957350099006E9E0D3957350028002C2
:1029E300D2359006E8E0D3957350099006E9E0C329
:1029F30095735002C235802A9006E8E0D395734060
:102A0300099006E9E0C3957340028002C23590063F
:102A1300E8E0C3957340099006E9E0D3957340025B
:102A2300D235229006EBE0903955F8282873804C74
:102A330085537380479000DFE0855FF0A4FFAEF01D
:102A430074081200398F738033856173802E856714
:102A53007380298568738024856973801F856A73F1
:102A6300801A856B73801585667380108565738006
:0C2A73000B856C73800690001EE0F5736C
:10395500022A31022A33022A38022A4C022A51024B
:103965002A56022A5B022A60022A65022A6A022A6C
:073975006F022A74022A7997
:102A7F009006ECE0FE9006EDE0D39E404B9006EB07
:102A8F00E0B404189006EDE0C395735002D236906F
:102A9F0006ECE0D395734002C236802A9006ECE034
:102AAF00C3957350099006EDE0D3957350028002E1
:102ABF00D2369006ECE0D3957350099006EDE0C343
:102ACF0095735002C236802A9006ECE0D39573407E
:102ADF00099006EDE0C3957340028002C23690065E
:102AEF00ECE0C3957340099006EDE0D39573400277
:102AFF00D236229006EFE090397CF8282873804C6C
:102B0F0085537380479000DFE0855FF0A4FFAEF040
:102B1F0074081200398F738033856173802E856737
:102B2F007380298568738024856973801F856A7314
:102B3F00801A856B73801585667380108565738029
:0C2B4F000B856C73800690001EE0F5738F
:10397C00022B0D022B0F022B14022B28022B2D02D3
:10398C002B32022B37022B3C022B41022B46022BF3
:07399C004B022B50022B55DA
:102B5B009006F0E0FE9006F1E0D39E404B9006EF1E
:102B6B00E0B404189006F1E0C395735002D237908D
:102B7B0006F0E0D395734002C237802A9006F0E04E
:102B8B00C3957350099006F1E0D395735002800200
:102B9B00D2379006F0E0D3957350099006F1E0C35D
:102BAB0095735002C237802A9006F0E0D39573409C
:102BBB00099006F1E0C3957340028002C23790067C
:102BCB00F0E0C3957340099006F1E0D39573400292
:102BDB00D237229006F3E09039A3F8282873804C63
:102BEB0085537380479000DFE0855FF0A4FFAEF064
:102BFB0074081200398F738033856173802E85675B
:102C0B007380298568738024856973801F856A7337
:102C1B00801A856B7380158566738010856573804C
:0C2C2B000B856C73800690001EE0F573B2
:1039A300022BE9022BEB022BF0022C04022C09025E
:1039B3002C0E022C13022C18022C1D022C22022C7A
:0739C30027022C2C022C311D
:102C37009006F4E0FE9006F5E0D39E404B9006F335
:102C4700E0B404189006F5E0C395735002D23890AB
:102C570006F4E0D395734002C238802A9006F4E068
:102C6700C3957350099006F5E0D39573500280021F
:102C7700D2389006F4E0D3957350099006F5E0C377
:102C870095735002C238802A9006F4E0D3957340BA
:102C9700099006F5E0C3957340028002C23890069A
:102CA700F4E0C3957340099006F5E0D395734002AD
:102CB700D238229006F7E09039CAF8282873804C5A
:102CC70085537380479000DFE0855FF0A4FFAEF087
:102CD70074081200398F738033856173802E85677E
:102CE7007380298568738024856973801F856A735B
:102CF700801A856B73801585667380108565738070
:0C2D07000B856C73800690001EE0F573D5
:1039CA00022CC5022CC7022CCC022CE0022CE502E8
:1039DA002CEA022CEF022CF4022CF9022CFE022D06
:0739EA0003022D08022D0D60
:102D13009006F8E0FE9006F9E0D39E404B9006F74C
:102D2300E0B404189006F9E0C395735002D23990C9
:102D330006F8E0D395734002C239802A9006F8E082
:102D4300C3957350099006F9E0D39573500280023E
:102D5300D2399006F8E0D3957350099006F9E0C391
:102D630095735002C239802A9006F8E0D3957340D8
:102D7300099006F9E0C3957340028002C2399006B8
:102D8300F8E0C3957340099006F9E0D395734002C8
:102D9300D23922AE2EAF2F74F5D39F74019E400813
:102DA300782E126FF0022EB0752F01752E00AE52E1
:102DB300AF53E546BE000DD39F40099000C1E0D359
:102DC300954740028023754700E546C39553F57345
:102DD3009000C4E0D395454008E5452573F545804B
:102DE300069000C4E0F5458002054790009DE0D3BE
:102DF3009561401CE55FC395604015AE52AF53E546
:102E030046BE00039F50099000C2E0D3954840029C
:102E1300806E9007DDE0A852B80004955350037507
:102E23004A009007DDE0A852B8000BD39553400643
:102E3300E5539007DDF0E54A7041E553C39546F548
:102E430073E573D3940540037573059000C3E0C322
:102E530095455007E573C3954540028009E545C391
:102E63009573F54580069000C3E0F5459000C3E0F7
:102E7300D3954540069000C3E0F5457548008002B0
:102E83000548E54A701690009DE0C39561500DE535
:102E9300462405A852B8000695534002800F9000BF
:102EA300B0E0F545754A0174789007DDF022AE2E47
:102EB300AF2F74E9D39F74039E4008782E126FF0EE
:102EC30002304F752F01752E00754532A23A402A04
:102ED3007545199000B0E075F002A4FFAEF0E54728
:102EE300BE0006D39F4002D23A0547754A03747861
:102EF3009007DDF075490002303EAE52AF53E54610
:102F03006F4E700302303EE546BE000DD39F40096D
:102F13009000C1E0D395474002800F754700E54A12
:102F2300C394035003754519800DE546C39553F5C6
:102F330073E5472573F54790009DE0D39561400EF7
:102F43009007DDE0A852B80007D395534002800CE8
:102F530005499000B0E0B54903754A00E54AB4035A
:102F630006A20DB3B34002800A0549E549B43C0308
:102F7300754A02E54AB402299007DDE0A852B80079
:102F83000ED395534009E5539007DDF07549009042
:102F9300009DE0C39561500975490074789007DD81
:102FA300F0E54A705A90009DE0D39561401CE55FBF
:102FB300C395604015AE52AF53E546BE00039F5024
:102FC300099000C2E0D39548400280087548007517
:102FD300454B8028E553C39546F573E573D39405B4
:102FE300400375730590009DE0D395614008E54863
:102FF3002573F5488006E5482406F548754900E53C
:103003004A701690009DE0C39561500DE546240576
:10301300A852B80006955340028003754A01E54A59
:10302300B4011875451905499000B0E0B549067516
:103033004A0275490074789007DDF0E54575F00A9A
:10304300A4FFAEF09007CEEEF0A3EFF022E56F9071
:1030530039F1F8282873900095E0700302327790D5
:1030630000CBE0B401028003023192900058E0B536
:103073005E02800302318F7E017F00E5BE126F9CEA
:10308300E5BD2FFF50010E8E5A8F5B7410126F9C9B
:10309300900083E08E048F05FF126F8C9007D2ECB3
:1030A300F0A3EDF074FFBC00039D500B74FF900779
:1030B300D2F8E4F0E8A3F0E56B600FE56BC394FE90
:1030C30050089000F1E06402600280649000DFE049
:1030D300B40B1F9007D2E0FEA3E0FF74E7126F9CCE
:1030E300E56B8E048F05FF126F8C9007D2ECF0A373
:1030F300EDF09000DFE0D3940B40089000C7E0644C
:10310300046002802B9007D2E0FEA3E0FF9007D477
:10311300E0FCA3E0FDEFD39DEE9C400D126FE89021
:1031230007D2EEF0A3EFF080079007D2E4F0A3F00C
:10313300900095E0B4021E9007D2E0FEA3E0FF905A
:1031430007DEE02FFF50010E74011200399007D201
:10315300EEF0A3EFF09007D2E0FEA3E0FF9007DECE
:10316300E0BE0008D39F4004D23D8002B23D9007E9
:10317300D3E09007DEF09000C7E064016006A23D53
:10318300B3B3400280069007D3E0F55F023275D2F5
:103193003D7E017F00E5BE126F9CE5BD2FFF500110
:1031A3000E8E5A8F5B7410126F9C900083E08E0416
:1031B3008F05FF126F8C9007D2ECF0A3EDF0E56B57
:1031C300600FE56BC394FE50089000F1E064026069
:1031D3000280649000DFE0B40B1F9007D2E0FEA3EF
:1031E300E0FF74E7126F9CE56B8E048F05FF126F8F
:1031F3008C9007D2ECF0A3EDF09000DFE0D3940BBA
:1032030040089000C7E064046002802B9007D2E07E
:10321300FEA3E0FF9007D4E0FCA3E0FDEFD39DEE17
:103223009C400D126FE89007D2EEF0A3EFF08007F9
:103233009007D2E4F0A3F0900095E0B4021E90074B
:10324300D2E0FEA3E0FF9007DEE02FFF50010E74F3
:10325300011200399007D2EEF0A3EFF09007D3E00C
:103263009007DEF09000C7E0640160069007D3E0AA
:10327300F55F8003755F00900091E07006756F0144
:1032830002305075BB18023845900091E07003027C
:1032930033FD7E017F00E5BE126F9CE5BD2FFF501D
:1032A300010E8E5A8F5B9000D7E0B4010F7E0F7F23
:1032B300FFAC5AAD5B126FE88E5A8F5B9000FCE057
:1032C300B40245AE5AAF5B900027E0FCA3E0FDEDEE
:1032D300D39FEC9E400A900027E55AF0A3E55BF0EC
:1032E300AE5AAF5B900029E0FCA3E0FDEFD39DEE67
:1032F3009C400A900029E55AF0A3E55BF0AE5AAF73
:103303005B74041200398F619000FCE0704CAE5A7C
:10331300AF5B900027E0FCA3E0FDEFD39DEE9C4064
:1033230009126FE88E5A8F5B8006755B00755A0031
:10333300AE5AAF5B7410126F9C900080E08E048FC6
:1033430005FF126F8C8C5A8D5B74FFBC0009D39DF3
:103353004005855B6180037561FE9000C7E0B401A1
:103363000280030233FBA20DB3B3500E90009BE027
:10337300A852B80005D39553500280719000D8E04D
:103383008561F0A4FFAEF074648E048F05FF126FA5
:103393008C8C5A8D5BE56B6016E56BC394FE500F06
:1033A3009000F1E0B402089000DFE0640B6002805B
:1033B30017AE5AAF5B74E7126F9CE56B8E048F05F3
:1033C300FF126F8C8C5A8D5BAE5AAF5B9007D2E0C5
:1033D300FCA3E0FDEDD39FEC9E4005855B5F800B76
:1033E300A23DB340069007D3E0F55F800BA23DB347
:1033F30040069007D3E0F55F800375610090009469
:10340300E07006756F0202305075BB1902384590A3
:103413000094E070030234B2E55ED3955140030299
:1034230034B0900025E0FEA3E0FFE565126FE09065
:103433000025EEF0A3EFF07E017F00E5BE126F9C46
:10344300E5BD2FFF50010E8E5A8F5B900101E07096
:1034530013740A126F9C74518E048F05FF126F8CC4
:103463008D658019AE5AAF5B740A126F9C8F048E00
:10347300057E017F95CDCCCD126E8A8F65E565D330
:1034830094644003756564900025E0FEA3E0FFE5C6
:10349300652FFF50010E900025EEF0A3EFF0900092
:1034A30098E0048E048F05FF126F8C8D6580037581
:1034B30065329000E4E07006756F0302305075BB0F
:1034C300130238459000E4E0604A7E017F00E5BEC8
:1034D300126F9CE5BD2FFF50010E8E5A8F5B740453
:1034E3001200398F669000E6E08566F0A4FDACF02B
:1034F3007464FF126F8C8D669000E5E08566F0A41E
:10350300FFAEF074FF8E048F05FF126F8CED9000F9
:103513007FF08003756600900092E07006756F047B
:1035230002305075BB17023845900092E0B4010297
:1035330080030235C07E017F00E5BE126F9CE5BDAE
:103543002FFF50010E8E5A8F5B9007DFE0601990BA
:1035530007DFE0149068FC12008CE493FC74019381
:10356300FDEDC39FEC9E400280069007DFE014F060
:103573009007DFE0C394B3501DAE5AAF5B9007DFF3
:10358300E0049068FC12008CE493FC740193FDEF5B
:10359300C39DEE9C400280069007DFE004F0900795
:1035A300DFE0FE9000B8E08E0088F0A4FFAEF07478
:1035B300648E048F05FF126F8C8D6780037567001F
:1035C300900093E07006756F0502305075BB1602CC
:1035D3003845900093E0B4010280030236697E010E
:1035E3007F00E5BE126F9CE5BD2FFF50010E8E5A82
:1035F3008F5B9007E0E060199007E0E014906A6643
:1036030012008CE493FC740193FDEDC39FEC9E4088
:103613000280069007E0E014F09007E0E0C394B363
:10362300501DAE5AAF5B9007E0E004906A6612004B
:103633008CE493FC740193FDEFC39DEE9C400280E8
:10364300069007E0E004F09007E0E0FE9000BEE0A3
:103653008E0088F0A4FFAEF074648E048F05FF1211
:103663006F8C8D68800375680075BB1F0238457EBB
:10367300017F00E5BE126F9CE5BD2FFF50010E8E4A
:103683005A8F5B7409126F9C74E68E048F05FF12C8
:103693006F8C8D6A90009AE07006756F0702305048
:1036A30075BB1502384590009AE070030237C47E5B
:1036B300017F00E5BE126F9CE5BD2FFF50010E8E0A
:1036C3005A8F5B74041200398F6990009AE0B40139
:1036D300159000EEE08569F0A4FFAEF074071200C8
:1036E30039EF9007D7F090009AE0B402159000EEFE
:1036F300E08569F0A4FFAEF07407120039EF90077C
:10370300D6F090009AE0B4030280030237A790003A
:10371300DBE0701CE569C394195002D22FE569D32D
:1037230094644002C22F9000BAE09007DAF08063FD
:103733009000BAE070349000EEE08569F0A4FFAE2B
:10374300F074FF8E048F05FF126F8CED9007DAF093
:10375300AE52AF53741EBE0006D39F4002D22FE574
:1037630061D394E54002C22F8029E569C3940A50CE
:103773000DAE52AF53741EBE0004D39F500280029D
:10378300D22FE561D394E54002C22F9000BAE090B6
:1037930007DAF09007DAE0C3940550067405900742
:1037A300DAF0C23E90009AE0B40414E569C39419B8
:1037B3005002D23EE569D394324002C23EC22F800A
:1037C300037569009000F1E07006756F08023050D0
:1037D30075BB14806D9000F1E060567E017F00E5BB
:1037E300BE126F9CE5BD2FFF50010E8E5A8F5BEF0B
:1037F300D39421EE940E4005756BFF8015AE5AAF3E
:103803005B7410126F9C74E38E048F05FF126F8C30
:103813008D6BE56B75F00BA4FFAEF09000DFE08ECF
:10382300048F05FF126F8C9007D4ECF0A3EDF080AA
:1038330003756B00900095E0600575BB1A800375F6
:02384300BB18B0
:1039F10002305902328C0234120234C702352C02D1
:0B3A010035D50236720236A90237D814
:05384500056FD2EC222A
:096FCE002582F5825002058322A0
:0F008C0025E050020583258250020583F582226C
:106F6B00EF2F500205832582F582E5833E2EF583B4
:016F7B0022F3
:106FE000CFC39FFF50011E22C3EF9DFFEE9CFE22E8
:086FF0000806B6000218062293
:0D6FAA00A3E004F07006120049E004F0229C
:0E003900048007C3CE13CECF13CFD5E0F6223E
:106E8A00BC000FBE0008ED8FF084FFADF022E4FED7
:106E9A00FF22BE000DEF60FE54F0606F20E7030290
:106EAA006F40EAC0E0EBC0E078017A0075F001EECD
:106EBA0020E710EF25E0FFEE33FE0AC5F023C5F008
:106ECA0030E7F0EA5407F9096A7A007B00600108A2
:106EDA00C3EC9E40167004ED9F4010ED9FFDEC9EA2
:106EEA00FCE5F0CA4ACA03F5F08005E5F003F5F0BF
:106EFA00C3EE13FEEF13FFD9D77908CACBCAD8D08D
:106F0A00EAFEEBFFD0E0FBD0E0FA22EC8FF084FC43
:106F1A00ED54F045F0C48FF084FEEDC454F045F012
:106F2A00C48FF084FDEEC4FE54F02DFFEE540F3CE6
:106F3A00FEADF07C0022790078008FF0EC7E08200C
:106F4A00E70DC3CD33CD33C933C9C833C8DEF084A6
:106F5A0049F9E5F08FF0BE00E6FD7C00E9FFE8FEA6
:016F6A002204
:0E6F9C00F88FF0A4FFE5F0CE88F0A42EFE22C0
:10000300EF8DF0A4F9A8F0EF8CF0A428F8EE8DF0B2
:06001300A428FEE9FF2213
:106F7C00600D782B026F86007830D8FED5E0F822B1
:106F8C00EEC0E07E00126E8AEFFDEEFCD0E0FE2239
:0C6FB700EEC0E07E00126E8AD0E0FE22E8
:03001B0002001EC2
:0300530002005652
:03009B00020071EF
:03000000026FD7B5
:096FD70075817575D0000244EBD0
:0B6FC300E5822FF582E5833EF5832276
:0A0049000582D5820215831582227C
:10001E00C0E0C0F0C083C082C0D075D000124419B9
:0B002E00D0D0D082D083D0F0D0E032E0
:10005600C0E0C0F0C083C082C0D075D00012441C7E
:10006600D0D0D082D083D0F0D0E032C0E0C0F0C093
:1000760083C082C0D075D00012449ED0D0D082D02A
:0600860083D0F0D0E0324F
:00000001FF
